S01A000066726565646F6D5F626F6F746C6F616465722E737265639E
S11300005028FF1F11040000EB040000AD4900005C
S1130010AF490000B1490000B34900002C060000BC
S1130020000000000000000000000000EB040000DD
S1130030EB04000000000000EB040000EB040000EF
S11300409B9200009B9200009B9200009B920000F8
S11300509B9200009B9200009B9200009B920000E8
S11300609B9200009B9200009B9200009B920000D8
S11300709B9200009B9200009B9200009B920000C8
S11300809B9200009B9200009B9200009B920000B8
S11300909B9200009B9200009B9200009B920000A8
S11300A02369000027690000CD4B0000D14B0000FC
S11300B09B9200009B920000C76B0000D76B00006E
S11300C0F56B00000B6C00001B6C00009B920000A1
S11300D09B9200009B9200009B9200009B92000068
S11300E09B9200009B9200009B9200009B92000058
S11300F09B9200009B9200009B9200009B92000048
S11301009B9200009B9200009B9200009B92000037
S11301109B920000FB8D00009B9200009B920000CC
S11301209B9200009B9200009B9200009B92000017
S11301309B9200001B2400009B9200009B920000F5
S11301409B920000D54B00009B9200009B92000004
S11301509B9200009B9200009B9200009B920000E7
S11301609B9200009B9200009B9200009B920000D7
S11301709B9200009B9200009B9200009B920000C7
S11301809B9200009B9200009B9200009B920000B7
S1130400FFFFFFFFFFFFFFFFFFFFFFFFFE3DFFFFBB
S113041072B60E480E49886000220023002400258D
S113042000260027B846B946BA46BB46BC4609482A
S1130430854609488047094880470948804762B68D
S113044000200021074A9047FEE70000000000005A
S113045000ED00E05028FF1F397B00003544000008
S11304607B440000493D0000000000000000000043
S1130470002A01D101207047F0B41F46034603242B
S11304802340002B09D00424E31A0170013008240E
S1130490E141521E26D05B1EF7D1042A1ADB13D089
S11304A0002F11D00C460D460E46102A02DB72C0F6
S11304B0103AFAE70C2A02DB32C00C3AFAE7082AAF
S11304C002DB12C0083AFAE7042A03DB01600430B5
S11304D0121FF9E7002A05D0017001300824E14118
S11304E0521EF7D1F0BC00207047FEE7252700001C
S11304F0000000004B270000000000002928000035
S113050077290000172800009B2800004B2A0000D0
S113051000000000012B00000000000085270000FF
S1130520000000005F2700009B2800005F2A0000F5
S113053000000000E12A000000000000B5260000D1
S113054000000000B92700000000000000000000C7
S113055000000000152B0000000000003B2B0000F1
S113056000000000772B000077290000CF2700004F
S113057000000000D7260000000000000001024631
S1130580853D0000133E000000000000313E0000E5
S1130590BF3E00007B400000AB4000000D41000066
S11305A019410000A1410000A94200000000000020
S11305B0453F0000374000008B3F0000D93D00005C
S11305C025420000000000000000000000000000C0
S11305D000000000570D00006D0D0000850D0000A7
S11305E0436F7079726967687420286329203230F8
S11305F031332D3230313620467265657363616C58
S1130600652053656D69636F6E647563746F722CD6
S113061020496E632E20416C6C2072696768747384
S11306202072657365727665642E0000299200005D
S11306300000024BE00500001000FF1F7C050000D5
S1130640D405000000000000759200007F920000B5
S1130650899200000000000000000000914A0000A0
S1130660D34A00002B4B00000000000000000000F3
S11306705F4B000001000000771200000000000042
S1130680000000008D2E0000BD2E0000FD2E000095
S1130690E32F0000000000001D3000002B69000063
S11306A06B690000116A00000000000000000000F7
S11306B04D6A0000E96A0000676B0000816B00006E
S11306C00000000000000000B36B0000534600006F
S11306D0DD4400000545000081450000BD450000E3
S11306E04145000052656164790D0A005472616EDF
S11306F07366657272696E670D0A000053756363F1
S11307006573730D0A0000004661696C7572650DAE
S11307100A000000EB3C904D5357494E342E3100F3
S113072002010100022000FF7FF0800001000100AF
S113073001000000FF7F0000000029313233344BF8
S1130740696E65746973205553420000F0FFFFFF22
S1130750FFFFFFFFFFFFFFFFFFFF000046534C209A
S11307604C6F616465722008000000000000000006
S1130770000000602C42000000000000412E0066D2
S1130780007300650076000F00DA65006E007400E7
S11307907300640000000000FFFFFFFF465345564E
S11307A0454E7E3120202012000000602C422C4255
S11307B0000000602C42020000000000426500724C
S11307C0005F0069006E000F00A8640065007800F7
S11307D00000FFFFFFFF0000FFFFFFFF012E006D81
S11307E0006500740061000F00A8640061007400DB
S11307F061005F006E000000650076004D455441C5
S113080044417E3120202022000000602C422C42F2
S1130810000000602C42000000000000412E005443
S1130820007200610073000F00256800650073000A
S11308300000FFFFFFFF0000FFFFFFFF5452415382
S113084048457E3120202022000000602C422C42AA
S1130850000000602C42000000000000422000491B
S1130860006E0066006F000F007272006D00610080
S1130870740069006F0000006E00000001530079ED
S1130880007300740065000F00726D0020005600B4
S11308906F006C00750000006D00650053595354DF
S11308A0454D7E3120202016000000602C422C4251
S11308B0000000602C42030000000000494E464F37
S11308C02020202054585420000000602C422C4248
S11308D0000000602C420500010000005354415404
S11308E05553202054585420000000602C422C42C0
S11308F0000000602C420600010000002E20202091
S11309002020202020202032000000602C422C4295
S1130910000000602C420200000000002E2E202067
S11309202020202020202010000000602C422C4297
S1130930000000602C420000000000004E4F5F4C9D
S11309404F47202020202020080000602C422C4209
S1130950000000602C420000000000007B00330017
S113096037003200300033004200460038002D00CA
S113097046004400380033002D00340033003200B8
S113098031002D0041003400430034002D003900B3
S11309904100390041004200460038004600420050
S11309A04300460044007D00000000002E2020206B
S11309B02020202020202032000000602C422C42E5
S11309C0000000602C420300000000002E2E2020B6
S11309D02020202020202010000000602C422C42E7
S11309E0000000602C420000000000004247007537
S11309F0006900640000000F00FFFFFFFFFFFFFF1E
S1130A00FFFFFFFFFFFF0000000000000149006E30
S1130A10006400650078000F00FF65007200560056
S1130A206F006C00750000006D006500494E444580
S1130A3058457E3120202020000000602C422C42AA
S1130A40000000602C4204004D00000075460000C8
S1130A50794600008B460000C946000000000000F3
S1130A600000000001000000040000005F230000FB
S1130A70B4060000C4060000200B000002000000C1
S1130A8001000000A32300009C060000AC06000047
S1130A90200B00000400000001000000D32300002C
S1130AA05C0600006C060000200B00001000000033
S1130AB000000000000000003C0B000000000000EB
S1130AC04C0B0000000000000000000000000000CB
S1130AD0000000000000000000000000CD740000D1
S1130AE00B7500003976000019770000B40BFF1F66
S1130AF0193400002B3200001D340000273400009C
S1130B002F33000031340000393400002B32000050
S1130B103D340000473400002F33000051340000FE
S1130B20257800002B7800009378000031790000CC
S1130B30297800003D79000005780000498A00000A
S1130B40478B0000378C00006D8C0000A38C0000E4
S1130B50C78C00004F8D0000E38D0000F38D000072
S1130B60F78D0000000000002DE9FF4B0C46434EBA
S1130B700178DFF80CB1317090464178717001252D
S1130B808178B170C178F1700179317141797171F5
S1130B908179B171C179F17100EBC5020BEBC5012B
S1130BA013780B706D1C53784B70062D00F06AF8A7
S1130BB0F2DB4FF00509052530788DF8000009EBCC
S1130BC0890170788DF801006918B0788DF80200F9
S1130BD00BEBC507F0788DF803006A4630798DF881
S1130BE004006D1E00F074F848408DF8070041467B
S1130BF000F085F800F0C6F89DF800003070012D73
S1130C009DF8010070709DF80200B07000F068F863
S1130C10F07100F044F8CFDAB9F10109CBD500F056
S1130C2088F80BEBC00204EBC00113780B70401C76
S1130C3053784B70062800F025F8F2DB2078A628BC
S1130C4004BF6078A62812D1A078A62804BFE07853
S1130C50A6280CD12079A62804BF6079A62806D13D
S1130C60A079A62802BFE079A628002001D04FF081
S1130C70FF3004B0BDE8F08B000000004809FF1FFE
S1130C805009FF1F93788B70D378CB7013790B7155
S1130C9053794B7193798B71D279CA7170479DF8EE
S1130CA0080038709DF8090078709DF80A00B87043
S1130CB09DF80B00F8709DF80C0038719DF80D003C
S1130CC078719DF80E00B8719DF80F00F8717047A7
S1130CD070798DF80500B0798DF80600F0797047C9
S1130CE09DF80300F0709DF8040030719DF8050034
S1130CF070719DF80600B0719DF807007047387850
S1130D008DF8080078788DF80900B8788DF80A0015
S1130D10F8788DF80B0038798DF80C0078798DF817
S1130D200D00B8798DF80E00F8798DF80F0068463B
S1130D3070473078207070786070B078A070F07868
S1130D40E0703079207170796071B079A071F079B8
S1130D50E0710120704710B5044600F087F820B117
S1130D602046BDE8104000F0C6B810BD70B500F0D4
S1130D7015F830B1324629462046BDE8704000F0EF
S1130D80C0B870BD70B500F009F830B132462946DC
S1130D902046BDE8704000F0C6B870BD04460D465C
S1130DA0164600F063B80268531C03601170704764
S1130DB00120704730B585B000F050F8002836D0D7
S1130DC04FF43040016800914168009B0191002B71
S1130DD082680292C068039008BF002903D1002AE8
S1130DE008BF002807D0DB4305D1C94303D1D14351
S1130DF001D1C0431BD0314CA06800688047A06873
S1130E000069D0F88C1011F1010F08BF4FF4826112
S1130E106A46002000F011F96946002200230024EC
S1130E2000253CC120B9264A0121117000E00020B0
S1130E3005B030BD80B52248007810B1002000F024
S1130E403BF9002002BD80B51D48007810B1002098
S1130E5000F03BF9002002BD00F0F2BD1948006823
S1130E60000E10F00F0018BF0120704715480068ED
S1130E70000E00F00F00012816BF022801200020F8
S1130E8070471148006870470F4908600B4989682A
S1130E9009694865704710B582B000228DF80020BA
S1130EA00A46064C014604F120002469646C6B4632
S1130EB0A0479DF8000000B1012016BD1000FF1FDF
S1130EC04A18FF1F248004407000FF1F10B5002142
S1130ED050F8212002F47F431B02140A43EA026300
S1130EE004F47F44234343EA126240F82120491C5E
S1130EF00429EDD310BD3248016841F4003101608A
S1130F007047F8B500F025F800F021F800F02AF851
S1130F102C4800F033F800F01AF8B4421CBF3046F5
S1130F20FFF7D4FF10E0F8B500F013F800F00FF865
S1130F3000F018F8244800F021F800F008F8B44252
S1130F401CBF3046FFF7C2FF00203861F1BD2046C8
S1130F50BCE704461D4F4FF0FF3038640D4616467B
S1130F602846B3E71A482968016069684160A9689E
S1130F708160E968C1601020B86070473860102053
S1130F803861B86C40F48030B8642168114801605D
S1130F9061680160A1680160E1680160B96CC9031E
S1130FA0FCD501693160016971600169B160006952
S1130FB0F060B86C40F48030B864284686E70000DE
S1130FC02C8004400D0210000C02100000100D4093
S1130FD000120D40E0170D402DE9F04196B0044693
S1130FE00D46164600F085FD804600271CE032467B
S1130FF003A92846FFF7B8FDA0B901A800F092FDA7
S1131000202205A901A800F093FD694601A800F07B
S1131010BBFD00980E99884204D105AA39462046A2
S113102000F06BFD40357F1C4745E0D3482103A801
S113103000F0C8FD16B0BDE8F081F8B514460FF213
S11310409C021C4E52F820504FF48072304600F03F
S1131050BDFD06F5807710222146384600F0B6FD26
S11310603846FFF778FE284600F028FD40F2F514D4
S1131070C0B9284600F038FDC8B93A46314628467A
S1131080FFF7AAFF284600F01DFD284600F024FDC6
S11310900028284602D100F022FD08E000F01FFDE0
S11310A00020F2BD022802D14FF4FA70F2BD2046AE
S11310B0F2BD0000700AFF1F80B50FF2200151F845
S11310C0200000F004FD002002BD80B50FF20C01E9
S11310D051F8200000F0F6FC002002BD00AC0D40E9
S11310E0DFF87409016841F440610160016811F49A
S11310F0406FFBD17047DFF864190A68904202D24E
S11311004FF0D04070474A68904201D20868704757
S1131110CA68904201D248687047CA68904234BF96
S113112088684FF0FF3070472DE9F04100F07DF8FA
S1131130DFF82C49DFF82C59DFF82C794FF00060E8
S113114000F06DFA00F071F82E683868C0B1D7F875
S11311500C8018F1010F04D03046FFF7CCFF404457
S113116028604FF01060206000F013F8D7F810806A
S113117018F1010F04D03046FFF7BDFF404428604A
S11311804FF08070206000F004F8386800B12E60E1
S113119040E2F8B54FF47A7000F08CFD04460D4639
S11311A000F07EFD4FF47A72A2FB046702FB057720
S11311B0841941EB070500F073FD8D4205D828BF63
S11311C0844202D240F29910F2BDDFF8A008006810
S11311D0C007F0D40020F2BDDFF89418D1F8D02174
S11311E0022A00D2704710B5DFF86C48226842F436
S11311F080420128226011D1D1F8D001A0B1216828
S1131200090E491C4843112828BF102021680902EF
S1131210090A401E41EA0060206005E0022803D16B
S1131220486CC0B200F03BFE20E0DFF848180A68C2
S113123040F2011002430A600A680242FCD170477E
S113124010B5DFF81448206820F48040206020683E
S113125040F0030020600A2000F035FD206840F4CF
S1131260804020602068800880002060206820F48E
S11312708040206010BDDFF80028DFF8003850B14E
S1131280012811D0022812D0032813D0042813D027
S1131290102813D014E01878002814BF002040F25E
S11312A095100860002070474FF0D040F9E7586867
S11312B0800AF6E71068F4E75068F2E75868F0E748
S11312C0042070472DE9F04FDFF8A4A70AF5E6776C
S11312D087B0386800B10120049000244FF47A707C
S11312E000F0E8FC81460498A0468B4650B100F01B
S11312F0D7FC04463868A9FB00230BFB0033CDE977
S113130002238846DAF84810DFF85457DFF85467A8
S113131001208840019000200090049838B100F02A
S1131320BFFC00F057F835D301D8904232D3FFF711
S1131330D7FEFFF77AFF3468B86888B1D7F8108011
S113134018F1010F04D02046FFF7D5FE4044306069
S11313504FF030602860FFF71CFF002837D134605D
S11313604FF040702860FFF714FF80BB00F098FC3A
S113137004464FF47A70A0FB092300FB0B33CDE93C
S11313800223884600F08CFC00F024F805D828BF1E
S1131390904202D240F2971019E0F06810F4F85F1E
S11313A0F0D0DFF8DC0600680090306E40F4803046
S11313B03066DAF84800C003009804D50199C043A8
S11313C00842AAD102E001990842A6D1002007B040
S11313D0BDE8F08F021B61EB0803DDE902019942CD
S11313E0704750B5DFF8882683B0526BA0F1D04027
S11313F00C46B0EB420FDFF8641604D24FF0D04035
S11314000090486802E0086800908868019000260F
S11314105DF82600DFF84C160860200001D0A047D4
S113142018B9761C022EF3D300205EBD2DE9F04FCF
S1131430DFF83C6681B0D6F8C4A114188046F06D7C
S113144089464AF08065002718B145F4803500E0EC
S1131450D044A04580F07D800120FFF7BDFEDFF879
S11314600076C7F8F880F06D10B9FFF75DFE06E06E
S1131470DFF810164046FFF7B4FFC7F8F880D6F837
S1131480D40198B1FFF7D1FED6F8E8B11BF1010FF2
S113149005D04046FFF72FFE5844C7F8F8004FF038
S11314A020603860FFF775FEC7F8F880FFF7BDFECF
S11314B0FFF716FED7F8580140F00060C7F858014E
S11314C0EFF3108072B6102159F8042BC7F84C21A1
S11314D0491EF9D10321C7F850113D60AAF140011A
S11314E0890810E059F8042BC7F84C21091F59F852
S11314F0042BC7F84C2159F8042BC7F84C2159F890
S1131500042BC7F84C210129C0F20880D7F85421D4
S11315109201E7D4D7F858215201F7D580F3108807
S1131520FFF737FE0220FFF757FED7F858014001B6
S113153002D54FF4CC770CE0F06D10B9FFF7C2FE82
S113154004E0DFF844154046FFF74BFF07003FF483
S11315507FAFFFF775FE384601B0BDE8F08F00009D
S11315602DE9F041804600204FF0D0450026DFF8F9
S1131570007506E00024032E0AD8DFE806F0020412
S113158006087C6B04E0BC6B02E0FC6B00E03C6C86
S11315902CB1DFF8D00405602846C04718B9651996
S11315A0761C042EE6D3BDE8F0812DE9F041054612
S11315B00120FFF711FEFFF7B7FDDFF8AC74DFF889
S11315C0A0443868E8B1D7F81880DFF8986418F1B7
S11315D0010F04D02846FFF78EFD40443060FFF72A
S11315E024FE00F01AF83560786808B1FFF79CFD16
S11315F0FF6917F1010F04D02846FFF77CFD381866
S11316003060FFF712FE4FF0007000F008F802207F
S1131610FFF7E2FD0020BDE8F0814FF0C0602060DC
S1131620B7E54FE610B5DFF86404FFF799FFDFF87C
S11316306004FFF795FF0446FFF702FE204610BD45
S11316402DE9F04105460120FFF7C6FDDFF81464DB
S1131650DFF81474DFF808443560FFF765FD386877
S113166090B1D7F8188018F1010F04D02846FFF77D
S113167042FD40443060FFF7D8FDFFF7CEFF3560F0
S1131680786808B1FFF750FDFFF7CFFD4FF0E06039
S1131690FFF7C5FF0220FFF79FFDFFF713FE044687
S11316A0FFF7CEFD2046BDE8F08170B5DFF8C043FA
S11316B0E16DB9B1626BDFF8DC63A0F1D0414D0894
S11316C0B1EB420F05F1D04005D2FFF7B9FF60B985
S11316D03068281806E0FFF7B3FF30B97068616B13
S11316E02818401ABDE87040AAE770BDF8B5DFF8C5
S11316F06813DFF8A423CA610A6822F0E0020A60D2
S113170000F10C02936C1BB10B6843F080030B6077
S1131710DFF85C53D66C012405F5BA733EB30E684A
S113172046F040060E6000F5D47006681EB10E68DF
S113173046F020060E601E6B0EB141F2010486686D
S1131740C768B6023F0406F4406607F47C173E43BC
S1131750076912683F0607F07C573E43344332B1B1
S1131760406800280CBF44F4007444F4807405F10C
S11317701000C26B032A08BF44F400449A6A0AB1F9
S113178044F48044DA6A0AB144F400544C62856D2E
S1131790C46DA4016D0104F0400405F020052C4340
S11317A0056EBE4A2D0405F4E0252C435460C46C38
S11317B0240404F480340C6284691B78240403F048
S11317C00F0304F4803423431360C26990F820307B
S11317D0120202F4706203F00F031A4303681B043D
S11317E003F440331A43CA60406BC0B200F057FBA5
S11317F00020F2BD2DE9F84F8146FFF7CAFCA84F3F
S1131800386840F080603860484600F067FB002884
S113181050D1974E9149706B984C00F1D0400860BC
S11318204FF0D048B26B10184860F26B1018886003
S1131830326C1018C8600021A0F1D04060600091A3
S1131840404609F13401042251F8043B13B1056800
S113185000951818521EF7D10098FFF7F1FC606844
S113186048B1F06D48B1706BF16B884202BFB06B48
S1131870316C884201D004207FE08A498A4A0A6098
S113188002234B600020002306EB8304874D646F22
S113189045F82040401C5B1C402BF5D30A60012016
S11318A048606D4E306840F4804030604846FFF731
S11318B01DFF20B1396821F0806139605DE0306836
S11318C0684F20F480403060386940F4807038619B
S11318D0D9F8780190B309F1340044460090042506
S11318E00098001D0090001F006828B33C60041994
S11318F009F5BC704068F8B14FF0000A09EB8A00A2
S113190000F5BE7BDBF80000B0B1FFF70DFCFFF77C
S11319108CFCFFF7E5FBDBF8100000F030F8DBF897
S11319200000B060FFF735FCFFF7CCFC20B90AF1EA
S1131930010ABAF1040FE1D36D1ED1D109F11C04DF
S11319402068C8B109F13409042559F8040B88B199
S1131950C7F800808044FFF7E7FBFFF766FCFFF75A
S1131960BFFB606800F00BF8A068B060FFF711FCE3
S1131970FFF7A8FC6D1EE8D10020BDE8F28F786562
S113198000207865786578657047F8B5050018BF5C
S113199015F0030044D1394C00202070284600F093
S11319A09DFA3F48016841F0806101602A4801685E
S11319B041F4804101600121416201680902090A80
S11319C041F0807101603A49C1610E2101614161B8
S11319D08161016841F00C010160016821F48041DA
S11319E00160FDB9334F4FF0D04635463068009062
S11319F00098FFF725FC3068B8420CD029482A49E2
S1131A000160022242602C4A026141F604424261B2
S1131A10016001214160FFF713FC3068B84201D036
S1131A200420F2BD124E4FF400722946304600F0F5
S1131A30DDF83046FFF7DEFE08B901212170F2BD62
S1131A400E480078704780B50C48007808B1FFF75D
S1131A50F7FB002002BD000000A00D4080A10D4056
S1131A6008A00D4000A10D40440EFF1F5CA10D40D5
S1131A70700CFF1F6CA10D40340EFF1F700EFF1F72
S1131A8000A20D4029110000C5120000AB15000092
S1131A902316000084A10D400040008004A10D40E5
S1131AA02C80044000A30D40F05AF05A10A30D40BE
S1131AB0000800806B716366130420084068C0F35B
S1131AC081007047016841F000410160704701687E
S1131AD049004908016070470068C00F70470168F9
S1131AE041F08001016070470068C00900F0010006
S1131AF070474068C0F30310704700EB811000F595
S1131B008070116801605168416091688160D1689A
S1131B10C160116901615169416191698161D16952
S1131B20C16170474FF0FF3101600021416070478F
S1131B30F0B585B004460D461646684600F0ECFA4A
S1131B4001208DF80B00206801901B4800900020B4
S1131B508DF80A00ADF808007EB100F026FB174F9F
S1131B606946384600F0A7FA32462946384600F05E
S1131B70D8FA3868019000F01EFB01982060606874
S1131B803018606005B0F0BD38B504460D462079C4
S1131B9010F0030007D0694600220A60C0F1040275
S1131BA02046FFF7C5FF206828600548016821F436
S1131BB08021016031BD0000B71DC1040020034035
S1131BC03C800440002200F005BB000062B38B0798
S1131BD008D0521E11F8013B00F8013B00F02480AC
S1131BE08B07F6D1830740F0208000BF103A07D35B
S1131BF030B4B1E83810103AA0E83810F9D230BC4B
S1131C00530724BFB1E80810A0E8081044BF51F8F6
S1131C10043B40F8043BD20724BF31F8022B20F8E0
S1131C20022B44BF0B7803707047083A07D3B1E81E
S1131C300810083A40F8043B40F804CBF7D25307A5
S1131C40E4E7000080B52B48016841F4000101601D
S1131C500020294908604FF0FF3128480161002223
S1131C6082610122C261826942F004028261826956
S1131C7042F00102826101600121C160816000F0D3
S1131C80CCF9C0001E49B0FBF1F000B901201D4998
S1131C90086001BD1848016841F002010160704705
S1131CA010B5194B19691A681C68A242FAD3D043BB
S1131CB0C94310BD13490968A1FB0001C00840EAEB
S1131CC04170C908704738B50446FFF7E9FF0D4A6B
S1131CD01268A2FB0423D20842EA4372141841EBAF
S1131CE0D305FFF7DDFFA942FBD301D8A042F8D307
S1131CF031BD00003C80044000700340007103408B
S1131D0040420F00980BFF1F0471034000F085B997
S1131D102DE9F0410646FFF793FE684C684D0246F4
S1131D202078002E5FD12968DFF8988161606649C8
S1131D308968096901F1680C9CF81C109CF8103042
S1131D402E681B09360F03F0010306F1010E002A69
S1131D5014BF5E4E5E4E01F0010183F0010739406D
S1131D6082F00107394206D04FF0A070B0FBFEF0BC
S1131D70C8F8000040E0B6FBFEF1C8F800109CF87B
S1131D801D10C94301F00F01491C0F468C468E46B5
S1131D902AB102270121BC464FF0040E05E023B10D
S1131DA0012101278C464FF0020E7F1E3F064B1E79
S1131DB007F0706747EA0373ACF101073F0507F4C6
S1131DC070073B43AEF101073F0407F470273B4320
S1131DD02B60B6FBF1F1C8F80010012100F00EF8F9
S1131DE00120207008E0012E08BF002A04D1002140
S1131DF000F004F860682860BDE8F081884281B092
S1131E004BD00129334824D102210173002102E07F
S1131E1000BF0099491C00910099B1F57A7FF7D36E
S1131E2030210170002AC17801F09F010CBF41F0FC
S1131E30200141F06001C1708179C906FCD4002001
S1131E4000900098B0F5FA4F27D200BF0098401CCC
S1131E50F6E7002908BF002A1FD1342101708179D7
S1131E60C906FCD50021017302E000BF0099491C9A
S1131E7000910099B1F57A7FF7D304210170C178FC
S1131E8001F09F01C170002002E000BF0098401CD7
S1131E9000900098B0F5FA4FF7D301B070470E499F
S1131EA00A681202120A012804D0022804D042F05F
S1131EB0407201E042F080720A607047580AFF1FC6
S1131EC0448004406001FF1F1000FF1F00D8B805C4
S1131ED0006CDC020040064000A00D40F0B5012576
S1131EE00024002600F134024FF4A063504908B9DD
S1131EF0012615E09769042F0BD3002051F8202008
S1131F0022F4E06241F82020401C0E28F6D304207D
S1131F10F0BD176807B90025976807B101242DB3F0
S1131F204B608B600B614B6186BB56684FF4E06578
S1131F3006B1CD619669022E12BF032E0B60CB60F1
S1131F409669032E0FD10B628B624B6200F5CE7043
S1131F508B61066806B1CB614668002E1FBF0B6318
S1131F60006800284B63506A00B1CD6274B1CB6144
S1131F700B628B62CB629069022804BF4B628B6157
S1131F80D06800B14B63506A00B10B630020F0BD10
S1131F902848294A01684908490001602748416BDB
S1131FA041F478514163016821F0406111430160BB
S1131FB0704710B51F48214C016841F001010160D0
S1131FC0FFF73EFD0028606B14BF20F4F05020F4AE
S1131FD0785060631A480168490049080160206824
S1131FE018490840206010BD1448016841F4E021FC
S1131FF00160016B41F4802101631148016841F0E3
S1132000004101601048017841F0800101700179BC
S113201041F002010171012070470C480C4A01682B
S113202000681268090F491CC0F30360514321E0A2
S113203000D0044000D000400000030404800440A9
S113204000700440FFFFF8F340210740448004403F
S11320506001FF1F0148024A04E000BF648004409D
S1132060006CDC020168006801F00101491CC0F346
S113207042005143401CB1FBF0F070470020704710
S1132080704700000B7A4A7A1B0703F0405343EA77
S113209082728B7A42EA8362CB7A1B0603F08073E6
S11320A01A4382600B68436042F00073836049689E
S11320B0016082607047E0B5164A136843F48023D8
S11320C013600A7B002A0A6800924A6801920DD1C3
S11320D04A7A02B102228DF808200A7A002A14BF33
S11320E0022203228DF809208A7A0AE000228DF860
S11320F008200A7A002A14BF022203228DF809203C
S113210000228DF80A20C97A8DF80B106946FFF772
S1132110B9FF07BD3C8004400FF248011022FFF7CD
S113212065BD03E011F8013B0370521E3AB111F092
S11321300303F7D103E051F8043B0360121F042AA0
S1132140F9D2002A03E011F8013B0370521EFAD1C0
S1132150704701688068C0F3017002282CBF080C26
S113216088B2704721100000FFFF0000000000004B
S1132170000000000160704772B60168491C0160EC
S113218062B601680029FCD10120704772B601686B
S1132190491E01E072B60021016062B6704772B652
S11321A009490020086062B6704772B606480168A3
S11321B0491C0160704704480168022900D2EAE71B
S11321C00168491E01607047800BFF1F62F30F22F4
S11321D062F31F4200B500BF1300964694461039BF
S11321E028BFA0E80C50FAD85FEA417C28BF0CC095
S11321F048BF40F8042BC90728BF20F8022B48BF6A
S113220000F8012B00BD000038B504463D4D002008
S1132210C5E90000C5E90200C5E904002862686256
S11322203948FFF747FDC5E906012046BDE83440BB
S11322300FF2550100F002B900F012B970B5314D3A
S11322400C46296A072904BF696A88421AD1FFF734
S11322505DFDC0EB0016D5E90001D5E90223101895
S1132260B6FBF0F00A2148434FF49661B0FBF1F05D
S1132270401D0A21B0FBF1F04FF496614843206001
S1132280002070BD012070BD2DE9F8430646FFF71C
S113229007FD1C4F0446386AD7E904598846421C96
S11322A0D7E90601651B68EB0909494502D82CBF2B
S11322B0A8420122012A3A6206D0042A08D0052A3B
S11322C00ED0072A0FD018E0C7E900487E6214E058
S11322D0D7E90001201A68EB0101C7E900010CE00D
S11322E0C7E9024809E0D7E90201201A68EB0101B5
S11322F0C7E90201304600F0B3F8C7E90448BDE875
S1132300F18300002009FF1F803801000901002823
S113231006D55F4A00F00F00801800F8041C7047CF
S11323205C4A8154704750F82130120423F470231E
S113233002F470221A430FE050F82100C0F3006049
S1132340704706E0120202F4E06242F0200203E069
S113235000BF120202F4E06240F821207047042812
S113236000D0704710B54C4C19B102290ED004D3DB
S113237010BD0020A063E06310BD4FF48070A06323
S11323804648016821F48041016010BD03220E21FA
S11323902046FFF7D6FF2046BDE8104003220F2158
S11323A0CFE7012800D0704710B53B4C11B102298A
S11323B004D010BD0020A062E06210BD02220B21F7
S11323C02046FFF7BFFF2046BDE8104002220A2145
S11323D0B8E7012800D0704710B5314C11B102297B
S11323E006D010BD002020616061A061E06110BDD5
S11323F0072204212046FFF7ABFF072205212046D0
S1132400FFF7A6FF072206212046FFF7A1FF20467B
S1132410BDE81040072207219AE780B50E211E4827
S1132420FFF78AFF48B11F480169080005D004205E
S113243088471D494FF0FF30086001BD10B50428DE
S11324400C460CD101213D20FFF760FF17494FF0E6
S1132450005008600A2200F016F81248046110BD0A
S1132460042800D0704780B511494FF0005008602F
S113247000213D20FFF74AFF002200F004F809493B
S11324800020086101BD0E2103484CE70000000054
S113249018ED00E000E400E000B0044094F00F40C8
S11324A000C00440A00BFF1FA0B0044004E100E002
S11324B084E100E0C16E11F1010F01BF016F11F160
S11324C0010F416F11F1010F02D042F6A20101E0A8
S11324D042F6A301C16270473EB504460D46684604
S11324E0FFF720FB04F10C004019001B6168A2688F
S11324F0051DA9423CBF5318984208D2421A6846A7
S1132500FFF716FB6068A1680818421B2946684655
S1132510FFF70EFB02A96846FFF736FB02983EBDA3
S1132520F8B51F4DA8680669F06A012442F6A301B4
S1132530884233D006F168070024B86858B3796834
S113254042428A4227D36A681368994221BF52687B
S11325504018401E82420FD2FEF77EFCD8B1686854
S113256000F1200278681168884214D35168BA686F
S11325701018401E81420ED34AF2C03106F16800A1
S1132580FFF7AAFF716F884206BF012442F6A0003C
S113259042F6A10001E042F6A400F0622046F2BD3A
S11325A01000FF1FBFF34F8FDFF8E406DFF8E426C7
S11325B0016801F4E06111430160BFF34F8F00BF74
S11325C0FDE7DFF8D416C968C968002008607047C1
S11325D02DE9F041DFF8C05682B0E86900248DF897
S11325E001404669002E62D0E968C9680A68012A78
S11325F04CD001F1080274680023091DA0470400AF
S11326001FBF42F21270844242F2137084424ED1D0
S1132610E868C168D1F80880B8F1000F47D04E6867
S1132620377837B1132F04DA806800EBC700083815
S113263000E00020086200281CBF006800281CD0AD
S11326402A699269694605F120009047040016D171
S11326509DF8000040B14FF4E750791EC840C00710
S113266058BF42F211740AD5EA68D268126A126835
S1132670414630469047002406E042F21074394641
S1132680204600F08DFA94B901200DE0086A48B1A3
S11326904168080003D00DF10100884704460CB1DD
S11326A0002001E09DF80100E968C968086020463F
S11326B0BDE8F68180B50178002000F071FADFF8FA
S11326C0D805C069416909698847022000F0E8FA21
S11326D0BDE8014066E770B5044601206168DFF893
S11326E0B85500F00FFBA8680069D0F8B4602178F1
S11326F0304600F055FA42F66810864209D1E8697E
S1132700416909698847022000F0CAFABDE87040AF
S113271048E770BDDFF88005C068C06814210C303C
S1132720FFF750BA10B50446606810B1012803D011
S113273005E000F09BFC03E000F047FE00E004200D
S1132740FFE72178BDE810402AE210B5DFF84825FC
S1132750126852690446A16860689047F1E710B5B1
S113276000F06EF8DFF83005C068C0686168016188
S1132770082101770020217800F012FABDE810400A
S113278001F0B1B830B583B0DFF80C45A56800217D
S1132790019100916B4681684068AD6801AAC9B295
S11327A0C0B2A847E268D2680021116100998A0882
S11327B0019900F009FA37BD10B5DFF8DC249268FE
S11327C0D26804466068A168C0B29047B9E770B5A2
S11327D004466068A568012805F2FF1607D128465B
S11327E001F083F918B1304601F07FF908B90425E6
S11327F00CE02846FFF7C9F80500DFF89C6402D115
S1132800306800688047B0680069456528462178CB
S1132810BDE87040C4E110B500F012F800F012F801
S11328200421017700208CE710B500F009F800F0CE
S113283009F8032101770020A168BDE81040DAE11E
S1132840044667E7DFF85004C068C068A168016106
S113285061684161704738B500F088F80021416132
S11328600161007F042804D128680069804704B905
S11328700446E868C068017F204600F091F942F2FE
S11328801270844208D1E868C068007F082804BF39
S1132890BDE8314001F09EB831BD2DE9FC4100F0A6
S11328A065F8016921B900202070FFF7D4FF5AE0D0
S11328B00121217006694769002000900123E8691D
S11328C0D0F814C0DCF804C06A4601A9E0475FEA06
S11328D0000805D0E8694169C9688847404603E0B3
S11328E0009830B942F21270FFF7B5FF0020207053
S11328F03AE0B04288BF30460090E868C068017F83
S1132900082913D10199C160009981610198009946
S113291001F02BF8804642F27D7080451CBF42F2E4
S1132920747080450BD14FF0000808E02B68019AC1
S113293000999B683846984780460098C7190098C4
S1132940361A06D0B8F1000F09D0E8694169C968A0
S113295088474046FFF77FFF0020207003E0E868C7
S1132960C068066147610020BDE8F681CA4D04468F
S1132970E868C06870472DE9F047C74D8AB004463F
S1132980E868C068016921B900202070FFF763FF7F
S113299057E00121217006694769C168027F212E31
S11329A02CBF4FF02008B046A9B1424601A8FFF75A
S11329B00DF9E869D0F814C0DCF808C001234246D8
S11329C001A9E047A6EB080606B1B0B3FFF743FF41
S11329D00020207035E0032A08EB070907D12B6893
S11329E05B6801AA414638469847824614E0102A9B
S11329F018BF4F46DDD190F81DA0FFF7D6FB39462E
S1132A002F69CDF800A04346FF6B01AA05F1200011
S1132A10B8478246FFF7CFFBBAF1000F4F46C8D044
S1132A20E8694569AD680123002201A9A847504619
S1132A30FFF711FF0020207004E0E868C068066119
S1132A40476100200AB0BDE8F08710B5924B1B68BF
S1132A50DB680446E268A1686068984771E62DE97E
S1132A60F04105468D4C6E68D5F80880E8688A49BF
S1132A70206000274968103130B10A68904223BFB2
S1132A804968491C81420427304601F02EF800B9F8
S1132A900427FEF7E1F940B1FEF7D5FFFEF78AF906
S1132AA008B140F2F717FEF7EFF92978384600F03D
S1132AB077F89FB96660002000F0F2F82068C4F847
S1132AC0088018B180F3088880F30988616840465B
S1132AD08847BDE8F041002000F0E2B8BDE8F0818D
S1132AE038B50446606801F000F808B9042005E030
S1132AF06568012000F0D4F8A068A847217819E09F
S1132B00654A10B5044602F120001269D269211DFC
S1132B10904716E638B5604D0446FFF746FB00F0D3
S1132B2024F86D6B04F10C02A8470546FFF743FB3C
S1132B3021782846BDE8344032E030B583B00446FD
S1132B4068460021002206C0534DFFF72EFB00F01B
S1132B500CF8AD6B6A46A8470546FFF72CFBA26844
S1132B606946284600F04BF837BD05F120002D6971
S1132B70A3686168704710B5FFF762FE4648C168F4
S1132B80C968A2680A6162684A6110220A77C0684B
S1132B90C068E16841770020A168BDE810405BE0AF
S1132BA010B584B0A02201908DF80020002200F01E
S1132BB06AF88DF80220029102228DF80320002386
S1132BC04469A4680C225BE010B588B0A72300F028
S1132BD03AF80020531C8DF8033006E06C4651F897
S1132BE0203004EB8004401CA3609042F6D300F034
S1132BF021F800231AE010B584B0A3222FE010B509
S1132C0088B0AF2300F01FF802238DF8033040B9D9
S1132C109008801C8DF80300029203A8FEF7E6FFDB
S1132C2001E000200290002300F004F86946A04768
S1132C3008B010BD1848C0699DF803104469A46821
S1132C4089000A1D70478DF80030019000238DF82B
S1132C5001308DF80230704710B584B0B0228DF881
S1132C6000200190012200F00EF8029100228DF85C
S1132C700220002302228DF803200C224469A46858
S1132C806946A0471FBD0448C0698DF801207047FC
S1132C900CED00E00400FA051000FF1FA409FF1F5B
S1132CA070B50446022C04D0002001F03CFB012C3A
S1132CB00ED00026114D06E04019C16889680A004B
S1132CC018BF8847761C1820704341590029F3D156
S1132CD074B9FFF76AFAFEF7DDFF01F0CEFB08498D
S1132CE0002008600120FFF713F8FFF762F962B6CD
S1132CF0BFF36F8FBFF34F8F70BD00BF640A000036
S1132D0008ED00E010B50C0003D1012000F01BF821
S1132D100446606800F0E9FE70B104F5707056492D
S1132D200068884208D1204600F01DF838B942F600
S1132D306B10BDE8104010E042F66A10F9E7204637
S1132D4000F06CF8F5E710B94FF420407047012803
S1132D500CBF4FF400300020704748498968096966
S1132D60C1F8B40070472DE9FF4104460020FFF785
S1132D70EAFF04F570758046102229466846FEF77E
S1132D8025FF444513D03D4FF86A46420020FFF723
S1132D90DAFF396A7A6A611A891A201A3140304096
S1132DA049428842A8BF0846029988420AD301983A
S1132DB0404507D1019429466846FFF78DFB0399E6
S1132DC0884201D0002000E0012004B0BDE8F08179
S1132DD02DE9F04104468846164688B031464046FF
S1132DE001F0AEFB0127A0B902E02C19A844761B20
S1132DF086B12025202E98BF35462A4621466846AE
S1132E00FEF7E4FE6A462946404601F07BFB0028B3
S1132E10EBD00027384608B0BDE8F081F0B5044691
S1132E2085B00020154EFFF78EFF0546102204F5ED
S1132E3070716846FEF7CAFE0298F16A4042494240
S1132E400840474201943A4629462046FFF7C0FF0E
S1132E5068B1B06800688047FFF762FB38B1394653
S1132E60204601F06DFB10B942F6681001E042F60D
S1132E70691005B0F0BD00006B6366671000FF1FAA
S1132E80C449EFF31080486072B6704738B5C24D3C
S1132E902B696C68DB6A2246042105F120009847FF
S1132EA02B69DB6A6A46012105F1200098472068F6
S1132EB000990818401E6060002032BDF8B5B64F76
S1132EC00446786B0D464042164600EA0401621A35
S1132ED0AA1852421040424207F120003F697F6C19
S1132EE06B46B84748B99DF8000008B16C20F2BDA4
S1132EF032462946204601F0BFFBF2BD2DE9F04FD2
S1132F0089B0924680460C4603AA00F01CF90600DC
S1132F105BD1A708BF00E41B4FF0FF300690079079
S1132F2005D0224607EB0A0106A8FEF74FFEFFF77D
S1132F30A7FF07EB0809984D4FB12E6976693B4608
S1132F405246414605F12000B047060009D144B17C
S1132F502E697669042306AA494605F12000B04784
S1132F600646DFF830B2DBF8040080F3108866BB55
S1132F709DF80C0058B3FFF783FF87B104A80290B3
S1132F80414605A80190534600F025F83A462E69BB
S1132F90D6F8288005F12000C047060010D17CB186
S1132FA004A8029006AB05A80190082200F013F8CB
S1132FB049462C69D4F8288005F12000C04706460C
S1132FC0DBF8040080F310880EB1304600E00020E6
S1132FD009B0BDE8F08FA8680069006DC0B2009028
S1132FE0704770B5044688B00D4600204DF8202087
S1132FF0401C0828FAD375B12026202D98BF2E46F0
S11330006A4631462046FFF779FF002804BF341989
S1133010AD1BF0D000E0002008B070BDF8B5044648
S11330200D46FFF72DFF5C4E5C4B37693F692A461E
S1133030214606F12000B847564F796881F310887D
S113304098B9B1680969096B79B1FFF719FFB068DC
S11330500069036D21463469646ADBB22A4606F1CD
S11330602000A047796881F31088F2BDF8B54A4C76
S1133070A16809696668326801F1580589692B6895
S113308000204F4293421ED16968914225D1FFF737
S1133090F7FE2269414992683E4D04F120009047B1
S11330A0696881F3108868B9A1680969096B39B145
S11330B0FFF7E6FE00F03EF8696881F3108808B96E
S11330C001212970F2BD9A4207D217EA030104D004
S11330D01046FFF7A3FF0028F4D16968494239403C
S11330E04A4271688A42EDD2481C811A1046BDE8F2
S11330F0F44093E770B5154682B000222A700A4660
S1133100254C2669766C01466B4604F12000B047D5
S113311078B99DF8001029709DF8001049B11D4D33
S1133120297831B900F006F808B16C2076BD012188
S1133130297076BDA06800692269016D126AC9B25E
S113314004F12000104770B50546134882B080682A
S11331500069006B0E46144600B101202070FFF791
S11331608FFE70428008800041426A462846FFF77D
S1133170C1FF0849496810B181F3108876BD81F315
S113318010889DF8000008B100202070002076BD52
S113319000000000600AFF1F1000FF1F6B66656BD4
S11331A038B50446B0484068012C0CBF00F1300526
S11331B000F12005FEF744FC18B9287240F295107E
S11331C032BD69461020FEF756F868BB009820B956
S11331D0286868604FF4C87032BD012C05D1B0F185
S11331E0806F08D94FF0806004E0B0F1006F02D91D
S11331F04FF000600090286800990918491E696022
S1133200012129727CB9994CA06069466868E06024
S11332100320FEF730F80098206069460420FEF78A
S11332202AF800986060002032BD70B500F07AF88A
S113323000B9C7E0324629462046BDE8704001F097
S11332401BBA2DE9F84301280C461546984603D1CC
S1133250204600F001F90446FEF7F2FB0028834FF4
S1133260834E08BF40F2951032D085B3307860B9F0
S11332703868401E044218BF40F2911028D1012042
S113328030700020B060746002E0F068A04219D190
S1133290B06839682A188A423DBFA9462919F160E5
S11332A0A1EB000980194A4641461030FEF78EFC16
S11332B0B0684844B0604C4439688842C844A5EBBF
S11332C00905D2D100F033F80028CED000E0002068
S11332D0BDE8F2837CB500F025F810B940F29510F2
S11332E076BD012C03D1284600F0B6F80546B40893
S11332F0A40006F0030608E001AA0421284600F011
S11333008DF80028ECD12D1D241F002CF4D136B1EA
S113331001AA3146284600F081F80028E0D100F0E7
S113332006F876BD04460D461646FEF789BB70B511
S11333304F4C20780025E8B14C4EA0683168884293
S113334005D0091A0019FF22103001F0C7F93268BC
S1133350606804F11001FEF769F80546002020704A
S1133360A0603DB93268606804F1100101F0EAF927
S113337000B124E0284670BD70B5FFF7D3FF00B953
S113338020E0012C03D1284600F066F805463748B2
S113339044686042054071420840464201E0361BE1
S11333A0651956B12846FEF780F938B921462846F2
S11333B000F020F80028F2D001E0002070BD40F2B7
S11333C0931070BD40F2951070BD80B5FEF738FBC8
S11333D010B940F2951002BDFEF724F948B923490B
S11333E08868C968091A491C00F004F808B140F259
S11333F0931002BD4942890889008008494280002F
S113340000E0091F31B150F8042B12F1010FF8D07C
S113341001207047002070470020C1E613460A4689
S1133420014600200DE713460A460146002051E7F5
S11334300A46014600209FE70120B1E613460A46EA
S113344001460120FDE613460A460146012041E7F4
S11334500A46014601208FE7034949680A6A096B55
S11334608018401A704700001000FF1F780EFF1FDD
S1133470880EFF1F10B504466068A168814211D20E
S1133480401A6060A1660FF2CD302060E08A28B156
S113349004F1280104F1380001F086F90120A0604C
S11334A0002010BD42F2787010BD10B50446002112
S11334B0DFF8D00501F078F9616A102204F12800E0
S11334C0FEF784FB606A00F01EF80FF2050017E0B7
S11334D010B50446DFF8B035606A4289A282C2683A
S11334E0921E626042689A4202D1017A022902DB8A
S11334F042F2757010BD00F006F80FF2150000BF1F
S11335002060002010BD04F13802102101F071B9CF
S113351010B5044682B0606A42686368A2610268BA
S1133520D21E9A42A26002D342F2767016BD02897C
S11335306AB1E28204F138024189C91E21660FF2A0
S113354039012160102101F054F9002016BD00203A
S11335508DF800006946DFF8342502F12000126975
S1133560926990479DF8000010B142F2817016BD37
S11335702046FFF77FFF16BD10B5044604F138025C
S1133580A068401EA0601021606A01F032F9206E2C
S1133590401E206604BF0FF235002060002010BDDD
S11335A010B5044604F12801A068401EA060DFF8AD
S11335B0D40401F0F9F8606A04F13802102101F032
S11335C040F92046BDE8104054E7000070B50546B8
S11335D01022A868696A461EAE6005F1380001F041
S11335E0B1F8002418B9DFF8A80428600BE0E88AD1
S11335F0401EE88280B220B1701EA8600120A86637
S113360001E04FF41E54204670BD38B50446E08AEC
S113361008B100F055F8DFF874542B68626A216E23
S1133620E06D9B689847A8B9A1682069491E884243
S113363003D328680069804760B900F046F800F0B9
S11336403AF80098616E884200D044E00FF20520F9
S11336502060002032BD38B50446E08A08B100F08D
S11336602FF8DFF8285400F030F82B68626AE06D18
S11336709B6810219847E8B9E06D1030E065206E32
S113368010382066112828BFDFF8080410D210B1C2
S1133690DFF804040CE028680069804750B900F0A2
S11336A00AF80098616E884200D014E00FF2A51069
S11336B02060002032BD694604F11C00FEF764BAA4
S11336C0626A1021104601F0BCB8616A102204F14C
S11336D01C00FEF72DBA42F27A7032BD10B50446D2
S11336E004F11C00FEF71EFA206E11282CBFDFF82F
S11336F0A403DFF8A40303E7DFF890331B68426EEA
S1133700016EC06DDB681847F8B50446B4F85A007A
S1133710C0F30321C0074CBF08250425E66D042926
S113372001D00420F2BDFEF740FD04F16002DFF891
S11337305C733C69646B2B46314607F12000A0475B
S11337400446FEF738FD002C14BF20460020F2BDCD
S113375070B5044642F27F76E56D284600F0C5F95F
S113376080B1606E04F11801A8470646012E03D10A
S11337702046BDE870407DE6022E03D100F0B3F888
S1133780002070BD304670BD10B500F15C01031D12
S11337901C684A685A60944202D242F2767010BDA4
S11337A00A7AD2070FD50A685C69A2420BD149682C
S11337B049B19960598A21B100F12801383000F0EB
S11337C0F3FF002010BD90F85A10C9075CBFBDE894
S11337D01040FFF74FBE42F27C7010BDB0F85A1093
S11337E08A070BD4CA070BD5C1F30320002808BFEE
S11337F0FFF73CBC012808BFFFF7E7BD0420704772
S1133800A24A126852695C3041680068104738B5B2
S1133810C46DB0F85A00C0F30320012804F2FF1568
S113382007D1204600F061F918B1284600F05DF98F
S113383008B9042032BD2046FEF7A7F80400934DD2
S113384002D1286800688047A8680069446520465A
S113385032BD0000D0B5044604F15806E08A5A2768
S113386008B1FFF72DFF616A30461022FEF7BEF95A
S11338700120815D7F18401C1028FAD33078F9B2FA
S1133880884202D042F27970D0BD71780A2942F29E
S1133890127025D8DFE801F01A060A0E26121A164D
S11338A0261C20002046BDE8D0406DE72046BDE838
S11338B0D04013E72046BDE8D0401DE72046BDE8D0
S11338C0D04045E72046BDE8D04087E70020D0BD82
S11338D02046BDE8D0409AE72046BDE8D04013E733
S11338E042F27B70D0BD70B56C4C70212046FEF75F
S11338F069F96B48654D2060FEF757FC2E69614CF1
S1133900B66B04232246302105F12000B0472E690E
S1133910B66B0423221D312105F12000B0472E6926
S1133920B66B042304F10802322105F12000B047EC
S113393005F120002D69AD6B042304F10C02332141
S1133940A847FEF738FC002054F8201011F1010FAD
S113395002D1401C0428F7D3042804D100200021FC
S1133960002200230FC4002070BDF8B504460D46A4
S1133970002000264B4FAE4217D03869C0F110002A
S1133980A91B09E079B13B69325DDA55761C3A69C5
S1133990521C3A61401E491E0028F3D1386100F0E0
S11339A005F810B9E7E742F27D70F2BD3B493D4AA4
S11339B04A620020CA682AB10B69934209D0581C94
S11339C0086101E08A6E12B9084609680847521E68
S11339D08A6670472DE9F0412C4C206800698047C5
S11339E000284DD1DFF8B48098F85900042833D169
S11339F008F15C052E68304600F077F807000BD01C
S1133A00FDF72AFA58B1FEF71EF8FDF7D3F900B115
S1133A100027FDF739FA17B940F2F71030E000201B
S1133A20FFF73EF998F85A00800710D56868686176
S1133A306168103158B10A68904223BF4968491C33
S1133A40814204201CD380F3088880F30988A86885
S1133A50B04742F27E7013E008280FD10220FFF72E
S1133A601FF9BFF34F8F1048104A016801F4E06159
S1133A7011430160BFF34F8F00BFFDE742F27B703B
S1133A80BDE8F0812013FF1F53544D501000FF1F59
S1133A90A1350000573600000B3600009812FF1FB6
S1133AA0AB3400000C13FF1F0CED00E00400FA051A
S1133AB038B504460D46FDF7C6FFFDF7C4F90020EE
S1133AC0FFF7EEF8A848A94A056044604FF4204186
S1133AD01160016881F3088881F309884068804790
S1133AE0BDE832400020FFF7DBB810B582B00028F3
S1133AF01EBF10F1010F9E49884201D1002016BD5E
S1133B006A46022100F066FD002418B90098007A84
S1133B1000B10124204616BD2DE9F04FDFF8549280
S1133B20954E85B0D9F80800006900F1680537465C
S1133B3009E0297C014205D07869FA6881695268F4
S1133B4038469047183738680028F2D10024A24636
S1133B50CDE9004A4FF47A70FEF7ACF8CDE90201E2
S1133B6008210020FDF797F930B94FF42040D0F830
S1133B7004B0D0F8008001E0A346A046FEF77EFA28
S1133B8000284AD15846FFF7B0FF07000ED0FDF7D2
S1133B9063F940B1FDF757FFFDF70CF900B10027B9
S1133BA0FDF772F917B1FEF7BBFC0746FDF742F9C2
S1133BB09FB3D9F80800006990F88600C00703D4C1
S1133BC041465846FFF774FF6A8A4FF6FF708242F7
S1133BD008BF41F28832DDE90201A0FB024A01FB81
S1133BE002AACDE9004AFEF75BF804468A46DDE9FD
S1133BF00001002908BF00280FD0FEF751F8021B6E
S1133C0061EB0A03DDE900018B4206D301D882424D
S1133C1003D341465846FFF74BFF374600E01837B9
S1133C2039680029E3D0287C0842F8D0F96809688B
S1133C30384688470028F2D0002FD8D009E0297CE4
S1133C40014218BFB74203D0F168896830468847FB
S1133C50183630680028F2D1384605B0BDE8F08F38
S1133C6030B583B0FEF79BFAFEF792F9414C216917
S1133C70496804F12000884721694048E06304F161
S1133C802000096C8847A06800688047FDF7DAFFC8
S1133C90FDF78EF878B3A06800692369D0F89850CE
S1133CA0DB6A6A46042104F1200098472369DB6A31
S1133CB001AA012104F12000984715F1010F15D044
S1133CC00098A84212D201990818A0F50070A842E1
S1133CD00CD34FF400712846FDF7DDF830B92846BF
S1133CE0FDF753FE40F29511884202D10020FDF702
S1133CF04CFEFDF7C9F8FEF758FAFDF7CBFFFEF7C7
S1133D005AFA0020FEF704F8FDF79CFF20680068CB
S1133D108047A0684068804700210020FEF7F2FF3A
S1133D20FFF7FAFEE061016919B109680A0018BFDA
S1133D308847E069416919B109680A0018BF8847D2
S1133D40E0680068804737BD38B5FFF789FF094C44
S1133D50E569E06840688047E868C1680800F8D011
S1133D6028468847F5E70000B009FF1F08ED00E08A
S1133D70110400001000FF1F640A00006400FF1F0C
S1133D807047000008B904207047DFF8B4150968CB
S1133D90090E01F00F010F290FBF4FF480210FF21C
S1133DA0746232F8111089020022026041604FF4FB
S1133DB08072012181604FF48051C160DFF8841565
S1133DC091F900309A404261C97881610021016112
S1133DD0016241620020704770B508B9042070BDCB
S1133DE0C4690FF2106165680C222846FDF7EEFEE7
S1133DF0DFF854650FF20861681C30601422A5686E
S1133E002846FDF7E3FE681C706002202060002055
S1133E1070BD38B5040001D1042032BDDFF82C2573
S1133E206FF03B4000F046F801D06B2032BD38E023
S1133E302DE9F04389B0164680460D4600F0EAF9B4
S1133E40049B00F0E3F904001BD1009D019F70194D
S1133E50461EB6FBF7F007FB106121B1401C784306
S1133E60461E00E07D19AE4217D32802000ADFF88F
S1133E70DC1440F010600860DFF8D404814502D0FF
S1133E806B2420465BE000F089F90446D8F8100062
S1133E90010018BF8047002CE4D0404600F043FAEC
S1133EA0EFE7204600F025FA0546204600F03BFAED
S1133EB0284632BD1060DFF89804814270472DE92E
S1133EC0F04389B004465FEA02080F461D4608BF66
S1133ED0042034D000F09FF9039B2A46394620463B
S1133EE000F054FA5FEA000929D1009FDFF85C640E
S1133EF002E00398C7192D1AEDB158F8040B70604D
S1133F0039020398090A042808BF41F0C06006D0AA
S1133F10082805D158F8040BB06041F0E060306027
S1133F20204600F0E6F981462069010018BF804769
S1133F30B9F1000FDDD0204600F0F5F9484609B08C
S1133F40BDE8F08370B5040018BF002A01D1042035
S1133F5070BDDFF8F803DFF8FC63CDB246EA05452F
S1133F60056010291568456002D01139032903D270
S1133F70082B04BF51688160204600F0BAF9054659
S1133F80204600F0D0F9284670BD2DE9F04389B0F1
S1133F905FEA0008914614BFB9F1000F04200E46F1
S1133FA01D4647D000F037F90698401E064208BF68
S1133FB005421AD1A919109C0020491E012C05D1D3
S1133FC0002E04BF691E07290AD10AE044B9FF295B
S1133FD007D9B6F5000F03D3DFF87C23914200D351
S1133FE0042038BBDFF864730DE0652022E07968B3
S1133FF049F8041B0699082904BFB96849F8041B49
S113400006998E196D1AADB13002000A40F0407065
S113401038602006069940F0FF1040F47F400429E0
S113402008BFB86002D0082908BF786000F0B6F86D
S11340300028DCD083E7F8B51546002818BF002D0A
S11340400C461E4601D10420F2BDDFF80073DFF8F0
S11340500C23E1B242EA0141396000F04AF958B94F
S113406079682960102C03D0A4F11101032903D22B
S1134070082E04BFB9686960F2BD002818BF002982
S113408001D104207047DFF8D802007800F0030261
S1134090022A08BF002005D000F0C00080280CBF11
S11340A00120022008700020704710B50A4600283D
S11340B018BF002A01D1042010BDDFF8A4321C78F7
S11340C0002104F00304022C1ED06FF03A41C3F81F
S11340D0021054781178240444EA0161947841EA86
S11340E00421D4782143C3F80610547911792404A7
S11340F044EA01619479D27941EA04211143C3F875
S11341000A1000F0F6F80146084610BD08B904206C
S11341107047DFF8502280E02DE9F04F89B09246D5
S113412080460C4600F076F8059B524621464046F0
S113413000F02CF978BB6A462146404600F03BF972
S1134140009C029E6042714208404542A54208BF5D
S113415075197E4F03E0AAEB0B0A5C447519BAF19A
S1134160000F17D0281BD346824588BF8346059885
S1134170BBFBF0F02102090A000441F0807140EA1F
S11341800920396040F0FF00786000F007F800284B
S1134190E1D000E0002009B0BDE8F08F4046A8E07F
S11341A02DE9F04389B080465FEA03090D461646BF
S11341B008BF042029D000F02EF8079B00F026F851
S11341C018BB009D109C614F05E007998A08761A78
S11341D009EB82094D19C6B12802000A40F00070AB
S11341E03860200640F0FF1040F47F407860D9F832
S11341F00000B860FFF7D2FF0028E6D0119901B1A2
S11342000D60129909B100220A6098E632462946E7
S11342104046BBE099466A46CDE042EA01414B4A3A
S1134220116066E02DE9F04180461E000D461746F8
S113423008BF042034D0042300F0A8F880BBD8F8C9
S113424014307A195F42C2F1000C07EA0C0CCCF16D
S1134250000C2F40ACEB07070021B7FBF3F7DFF8A6
S113426008C10AE0DCF800E0203C6FEA0E0E2EFAEA
S113427004F4E40748BF491C5D1995420AD2B5FB12
S1134280F3F4202C38BFDCF804E0EED3D8F818E0BF
S11342907445E7D319B1B94234BF02210121317009
S11342A0BDE8F08100000000002818BF002A01D1F9
S11342B00420704709291AD8DFE801F00509090B21
S11342C00D0F11131517C068106000207047406867
S11342D0FAE78068F8E70068F6E70120F4E7406948
S11342E0F2E78069F0E7006AEEE7406AECE76A20EB
S11342F0704710B51D4C7021217000F03BF888B94F
S113430011490968204688472078810601D567202D
S113431010BDC10601D5682010BDC00701D56920B4
S113432010BD002010BD38B50400200000F022F8B4
S11343300500002D03D10E4803494968884731BD63
S11343404C80044028000240680AFF1F0400024019
S11343506B66656BFFFF004300048000FFFF0041B4
S113436002000240FFFF004018000240000002402B
S113437004F0014008B904207047C06920B1006806
S1134380022801D1002070476D20704708B904202D
S113439070475B1E194208BF1A4201D0652070475E
S11343A00368994221BF4068C0185118884234BF3D
S11343B066200020704770B505000E46144601D1F2
S11343C0042070BD20212046FDF7FCFB2868301A2C
S11343D02060E8686060A9686868B0FBF1F0A060DC
S11343E00420E0601020206160610420A061E0618D
S11343F0002070BD8021017002780A42FCD0704711
S11344000168F02212040A430260BFF36F8FBFF306
S11344104F8F704708001000180020003000400043
S113442060008000C000000180010002000300045D
S11344300006000080B51B491B4808601B491C4846
S1134440421A1C4888421CBF002AFDF7BFFB1A48C9
S11344501A49091A18BF00F03BFA19481949091AF0
S113446018BF00F035FA18491848421A04D0BDE8BC
S113447008401748FDF7AABB01BD16484FF0FF31AD
S1134480016041608160C160016141618161C1611C
S11344901148016041608160C160016141618161D5
S11344A0C161704708ED00E000000000A88E000024
S11344B0289200000000FF1F2009FF1F4C18FF1F57
S11344C00004FF1F2009FF1F049300000493000051
S11344D04C18FF1F80E100E080E200E070B50D00A1
S11344E082B00446164601D1002076BD6A4600F02B
S11344F071F830B9009BDB685B6832462946204678
S1134500984776BD70B50D0082B00446164601D1B9
S1134510002076BD00F07FF800B14CE000F047F8D1
S113452068B9009BDB689B68324629462046984759
S11345304E49002806BF009AD26800220A6076BD60
S113454038B504460D466A4600F044F8A0B9009810
S1134550C068406908B9662032BD2946204600F08B
S11345605AF810B142F2D87032BD009AD26852693A
S113457029462046904732BD002DFCD1002032BD93
S113458070B50D0082B00446164601D1002076BDF8
S113459000F041F800B10EE000F009F830B9009BDA
S11345A0DB68DB68324629462046984776BD6A4672
S11345B0294620460EE042F2D87076BD10B52B4C49
S11345C02168002029B109690A0002D08847002126
S11345D0216010BD70B542F2D873D2B1244C646826
S11345E0146011B915E01034146014688CB1256896
S11345F0002D04BF6668002E01D1E6684EB1A842C2
S113460024BF65688542EED30818401E854228BF42
S11346100023184670BD70B50918491E0022144BBA
S11346209C685D682469160104EBC204583475590A
S113463066682468AC4208BFAE4205D0864228BFF3
S1134640A14201D3012070BD521C022AE8D30020EC
S113465070BD10B50648446804E00068010018BF46
S113466080471034E0680028F7D110BD940BFF1F79
S11346701000FF1F00F030B9134680B50A4601460A
S11346801846FDF7A3FA002002BD70B510F0030F21
S11346900C46154612D0B0F1005F0FD22118491E06
S11346A0B1F1005F0AD3C0F1005632462946FDF746
S11346B08DFAA21B71194FF0005001E022462946E1
S11346C0FDF784FA002070BD10B514460A46214651
S11346D0BDE810400123FBF7CBBE000062F30F22BC
S11346E062F31F42401810F0030308D0C91A1FD305
S11346F0DB0748BF00F8012D28BF20F8022D130066
S113470030B414461546103928BF20E93C00FAD8C5
S1134710490728BF20E90C0048BF40F8042D890050
S113472028BF20F8022D48BF00F8012D30BC704787
S1134730C91818BF00F8012DCB0728BF00F8012DB8
S1134740704700000300002013F0030F09D0521E2D
S113475022BF13F8010B11F801CBB0EB0C00F3D01E
S11347607047121F22BF53F8040B51F804CB604565
S1134770F7D0121D0AD200BA9CFA8CFCB0EB0C00E4
S113478038BF6FF0000088BF01207047521E22BF5F
S113479013F8010B11F801CBB0EB0C00F6D0521C4E
S11347A008BF10467047000070B50D46424C30B14A
S11347B00146102204F11000FDF708FA06E004F1A6
S11347C0100000210022002300264EC02DB110222B
S11347D029462046FDF7FAF905E0002000210022D1
S11347E000230FC4103C04F11000BDE87040FCF736
S11347F0B2BA2DE9FF4100F058F81EE000F050F87D
S113480000983168484000906A46019871684840B1
S1134810019010340298B168484002907F1C0398BC
S1134820F1684840039006F110016846FCF79EFACF
S1134830684600F043F8103E10354745DED3BDE826
S1134840FF812DE9F04188B000F02FF823E0102219
S1134850214604A8FDF7BAF900F022F86A4606F1E9
S113486010016846FCF78EFA0098316848400090C1
S1134870103401987168484001907F1C0298B16817
S113488048400290F16803984840039004A800F05F
S113489015F8103E10354745D9D308B0BDE8F0816E
S11348A0102221466846FDF791B9044615464FEAA1
S11348B011180027004E7047380AFF1FB0E80E1089
S11348C0A6E80E10102269462846FDF77FB90000BD
S11348D00022FFF707BF00001D480068000B00F02E
S11348E00F00C01E082830D8DFE800F005080B0EC2
S11348F01114172F1A004FF4804013E04FF4C040F6
S113490010E04FF400400DE04FF440400AE04FF453
S1134910803007E04FF4C03004E04FF4003001E091
S11349204FF480200321421E10420A4A18BF02217C
S113493052684B1CB0FBF3F0C0F1005342F8103F37
S11349406FF0604301FB003050600020704700BFEF
S1134950007004401000FF1F02280ED80FF224023A
S113496080560122012900F01F0102FA01F10CBF57
S1134970024A034A400942F82010704700E100E06F
S113498080E100E01A1B4100BFF34F8F0548064A3F
S1134990016801F4E06111430160BFF34F8F00BF70
S11349A0FDE700000CED00E00400FA05ECE7EBE79E
S11349B0EAE7E9E702280ED80FF224028056012222
S11349C0012900F01F0102FA01F10CBF024A034A57
S11349D0400942F82010704700E100E080E100E067
S11349E018194A0004280ED80FF224028056012216
S11349F0012900F01F0102FA01F10CBF024A034A27
S1134A00400942F82010704700E100E080E100E036
S1134A101E1F202122000000002101807047F0B5F4
S1134A2085B004460D4616466846FDF775FB002022
S1134A308DF80B002088019041F2210000900020A5
S1134A408DF80A00ADF808008EB1FDF7AEFB0E4FED
S1134A5069463846FDF72FFB324629463846FDF7AE
S1134A6060FB3846FDF775FB0190FDF7A4FB019848
S1134A70208005B0F0BD008808800448016821F456
S1134A808021016070470000002003403C80044006
S1134A9040684A49405C70474849CA6842B18A68DC
S1134AA013780370501C8860C868401EC860704743
S1134AB00021017070475A2807D1404A01238B54C2
S1134AC00FF2090151619169084770473B498969AF
S1134AD008477FB5394DA96104460FF2FC006168AF
S1134AE050F82160684600F0F7F801208DF80800BE
S1134AF08DF8090002213248286132486861A268B1
S1134B00606890476946304600F097F82E49304671
S1134B1000F014F960680121FFF71EFF616849196C
S1134B200120087104B0002070BD70B50546234C07
S1134B3068680119097989B10FF29C0151F8206064
S1134B400021FFF709FF304600F0D2F86868AA6830
S1134B5000219047696809190020087170BD174841
S1134B608160C260C1680029FCD10020704770B523
S1134B7004460FF2640082B050F82450E86A000141
S1134B800BD54FF0006007E03169684688479DF80F
S1134B90000068634FF00070E862E86A074E800125
S1134BA0F2D4E86A800308D5A86B4FF40031E962B7
S1134BB021467269C0B29047F3E773BD9800FF1FA6
S1134BC0994A0000B74A00000000020A0020CEE71C
S1134BD00120CCE70220CAE700C0024000D0024016
S1134BE000C00A40010C01F1804101F58E2101232E
S1134BF00A6803FA00F0104308607047002901684E
S1134C0014BF21F4804141F48041016070470021C8
S1134C100FF2140252F82130834202D0491C0329B6
S1134C20F8D308467047000000C0024000D002409C
S1134C3000C00A4001212046E0E738B504460D468D
S1134C40FFF7E5FF00F043F8FFF7F4FF00F088F802
S1134C500122206840004008206020680840297B29
S1134C6040EA8170A97B40EA8160697B40EA016087
S1134C70E97B00F019F80121204600F054F8287867
S1134C8004EB8000C1686A6800F014F82A7A92067E
S1134C9002F0806211436A7A520602F000721143F4
S1134CA0C16000F00FF831BD090201F440710843FE
S1134CB020607047521ED20621F0FE4102F0F042FD
S1134CC011437047206840084000206070470FF28D
S1134CD0A00151F8200085E70021017008214160FE
S1134CE0002101724172017341738173C173704772
S1134CF010B504460021206800F034F8FFF79BFF4C
S1134D0000F02CF80FF2680151F82000010C01F1B9
S1134D10804101F58E2101230A6803FA00F022EA9A
S1134D200000086010BD0368090401F47C11012A25
S1134D300CBF194323EA0101016070478A0103D5BE
S1134D40026B22F0807202638A0303D5026B22F4A1
S1134D5080320263026B114301637047204656E7B9
S1134D602068024940F0010020607047FFCCFFBA80
S1134D700C003C100D003C100C003010010C01F133
S1134D80804101F58E2101230A6803FA00F01043E3
S1134D9008607047010C01F1804101F58E21012367
S1134DA00A6803FA00F022EA00000860704700294C
S1134DB0817814BF41F0800101F07F018170704758
S1134DC000210FF2F00252F82130834202D0491C34
S1134DD00429F8D3084670474A0603D5827842F07E
S1134DE040028270890603D5817941F020018171E6
S1134DF07047C1788279520648BF41F48041807976
S1134E00C00648BF41F480510846704738B504468F
S1134E100D46FFF7D5FF00F030F8A87A10B102284C
S1134E2004D00DE0E8884000207009E0E8884000E4
S1134E30207028894000E071607940F008006071BA
S1134E40A078A97800F0FD0040EA4100297840EA02
S1134E50C110A0706079297900F06F0040EA011058
S1134E60697840EAC110E97800F001F831BD00F03A
S1134E70DF0040EA4110607170470FF2480151F8B9
S1134E8020007BE710B504460021FFF790FF204681
S1134E90FFF796FF0FF22C0151F82000BDE81040F7
S1134EA078E70021817241708170C1700171012124
S1134EB001707047006006400070064000600E40BC
S1134EC000700E400600341007003410060028104D
S1134ED00700281000210FF2C81252F82130834233
S1134EE002D0491C0529F8D3084670472DE9F04142
S1134EF00D460446286800260146B046042303FBF9
S1134F0000FCB2FBFCFC1FFA8CFCBCF1000F08BFD8
S1134F104FF0010C0CF101070CFB03FE5F43B2FBE5
S1134F20FEFEB2FBF7F7AEEB000EC71B77453CBFA6
S1134F30BE460CF1010C714502D371461E46E04693
S1134F405B1C212BDBD36422B0FBF2F000EB4000AE
S1134F50884238BF40F221504ED32046FFF7BAFFB3
S1134F6000F05EF810430860311FA06820F4402070
S1134F70A06004292068DFF8241138BF40F4003011
S1134F800840711E090601F0F85108434FEAC84170
S1134F9050EAD1402060206820F000502060A068D2
S1134FA020F01000A060A06880088000A060A068C5
S1134FB029790843A06020686979490320F40050E6
S1134FC001F4005108432060A979E87941EA0040DE
S1134FD0E061A06940F08800A061A06940F440400D
S1134FE0A061A068297A09B140F40020697A09B166
S1134FF040F48020A0600020BDE8F08180B5C16944
S113500011F47F4FFBD141684902FCD50021816036
S1135010FFF760FF00F004F822EA0000086001BD19
S11350200FF2900151F82000010C01F1804101F5CB
S11350308E2101230A6803FA00F070474FF4E1312E
S113504001600021017141718171C171017241726C
S1135050704710B50A02036802F440442343036016
S113506002F4407283691A438261090A826842EA3F
S11350700121816010BD41688069000C00F0C3000B
S11350800843704705E043681B02FCD511F8013B57
S1135090C36013465A1E002BF5D1704700E0FFE0B1
S11350A000400C4000500C4000600C4000700C406C
S11350B000600D4004002C1005002C1006002C107C
S11350C007002C1016002C1070B5424E01243068D5
S11350D0491E1546082900F10C024CD8DFE801F0FE
S11350E0051423424228424B4000696811F1010F24
S11350F018BF00290ED0D168012912DB90F84610A0
S113510001290ED118300AE0696811F1010F18BFA6
S1135110002901D1002070BD116114701430FDF715
S113512035F8002427E024212030FCF74BFD22E051
S1135130A978002904BFE978002904D12978012934
S113514008BF547017D06A6829462030FCF73EFD2A
S113515030686968C16104731430FDF717F80AE018
S1135160052408E000211430FDF704F8306800211C
S11351701830FCF7FFFF204670BD38B50C46002000
S1135180012C0DD1134D286880F8461000F120023F
S113519080682423022100F0C8F9296881F8474077
S11351A032BD002051B90B48006880F8482000F156
S11351B0200280682423022100F0B7B97047054912
S11351C0086000207047034908600020096888606F
S11351D070470000840BFF1F10B5134601200BB964
S11351E0032010BD00225A745A6832B11468220098
S11351F003D00A4601211846A04710BD10B5134636
S113520001200BB9032010BD00229A745A6832B1F0
S11352101468220003D00A4602211846A04710BD94
S11352202DE9FF410446002561688968227B4B799A
S1135230012093424ED3096800294BD001EBC201EF
S11352400839002200E0521C0B789A4242DA4B687B
S11352500C2606FB02331E78032EF4D194F80EC0FC
S1135260002100E0491C1A7A914205DA5A680E01BD
S1135270B75C6745F6D1B518D978617355B3A560A5
S11352804FF00008974E984F07E0039402AA206855
S1135290694600F059FA08F101082979884519DAB4
S11352A000208DF80400A86810F828008DF802008A
S11352B0C009A96801EB880101284988ADF80010EC
S11352C0A96801EB880149788DF803100CBF029797
S11352D00296DAE704B0BDE8F08138B5044601204F
S11352E0A16861B1002506E0886810F825102068DF
S11352F000F047FA6D1CA1680A799542F4DB32BDCF
S113530070B504461546012084B0002D14BF002C4E
S113531003200BD0491E052908D8DFE801F05A0301
S113532008182E44002121736174A174B9E06168E6
S113533000291EBF217B2A788A42F7D011B120466A
S1135340FFF7CBFF287820730020A07311E0616879
S11353500029EBD02988627B0D460904B2EB116F5A
S11353600AD1A17BEDB28D4206D02046FFF7B5FFEE
S1135370A5732046FFF754FF93E0616800291CBF22
S1135380A1680029F8D00026A26811798E42F3DAC8
S11353909268297812F82620914204BF206800F010
S11353A008FA761CF0E7616800291CBFA16800298F
S11353B077D00026A26811798E4272DA9268297831
S11353C012F82620914204BF206800F0FCF9761CF4
S11353D0F0E729680A7802F01F02012A02BF0A795D
S11353E0637B9A425DD14A78012A20460AD0022A78
S11353F013D0032A1AD0092A22D00A2A40D00B2A11
S113540045D04DE04988090A8DF808106A46296894
S113541049888DF80910032120E063681B6804F1B2
S11354200F020421984704F10F0107E063681B6829
S113543004F110020421984704F11001696030E07E
S11354404988090A8DF80810296849888DF80910D7
S1135450297B59B1A96801916A46092163681B68CF
S11354609847009969600199A9601AE069680091F8
S11354706A46A9680191062163681B68984710E091
S11354804988090AE17329688A1C072104E04988CC
S1135490217404F11002082163681B68984700E036
S11354A0052004B070BD70B50C46154600211423C8
S11354B00E4A03FB0126326822B1491C0129F7DB9D
S11354C0022070BD314600F01CFA50B9306808B9AA
S11354D0032070BD002030737460FF20B0732E6011
S11354E0002070BDFD510000D9510000A406FF1F2B
S11354F010B5040001D1032010BDFFF7EEFE00211A
S1135500216061602173A17310BD10B5040001D145
S1135510032010BD607C08B1022010BD206800F09B
S113552001F908B90121617410BD10B5040001D15D
S1135530032010BDA07C08B1022010BD206800F03B
S1135540F6F808B90121A17410BD000010B5044695
S113555000F0DCFA0020206084F88D0000F0E0FA0E
S1135560002010BD38B508B9032032BD446844B1E9
S113557000680D0602D5A468A04732BDE468A047C0
S113558032BD062032BD08B903207047436813B109
S113559000685B691847062070473EB504460A7ADE
S11355A0D5090120102A02F00F0319D100220B2182
S11355B02046FFF7E8FF04F18C00022181700022ED
S11355C000210170002004EBC001401C1028CA60B7
S11355D00A61F8D3A36801212046984700203EBD04
S11355E0082B11D245EA430204EBC203DA685AB12C
S11355F00868009048680190487A8DF80800694668
S11356001A69DB68204698473EBD002918BF002868
S113561001D1032070478268002A18BFFFF7BDBF7D
S1135620012070472DE9F04107461400884608BF61
S1135630032053D000F06AFA294D286805F18C063E
S113564030B171788F4203D100F06AFA01273FE04C
S113565018B100F065FA02273AE0777000F060FABA
S11356600020C5F8088077703070002205EBC00177
S1135670401C1028CA600A61F8D3012F19D80FF210
S1135680F8106860174800281CBF174800280BD082
S1135690164800281CBF1648002805D015480028C5
S11356A01CBF1548002809D12846FFF74FFF0720E3
S11356B014E02846FFF74AFF06200FE02A46294651
S11356C0384600F05AFC070004D0284600F019F8C8
S11356D0384603E00220B07025600020BDE8F08168
S11356E01406FF1F7B5F0000E95F000023600000D9
S11356F09160000037610000796100000022002100
S113570041E710B5040001D1032010BD616821B147
S1135710206849688847002060602046FFF716FF2C
S1135720002010BD01F00F0141F080011AE701F0E3
S11357300F0117E708B903207047426812B10068E7
S1135740126910470620704710B508B9032010BD30
S1135750002918BF002A12D08B7803F00F04082CFC
S11357600DD2640044EAD31300EBC3031468DC6075
S113577052681A610A46BDE81040022103E704207A
S113578010BD73B5044601F00F05CE090CB9032012
S113579076BD01AA0321FFF7F6FE082D07D246EADB
S11357A0450104EBC1010022CA600A6176BD0420F0
S11357B076BD02B501F00F01082902D26A46042120
S11357C00BE0042002BD02B501F00F01082902D24A
S11357D06A46052101E0042002BDFFF7D4FE02BDA4
S11357E00000000010B501230AB9042010BD891E71
S11357F0062900F18C0417D8DFE801F004060E1026
S1135800080A12000C210CE00D210AE0A07800E047
S113581020780023107007E0062102E0072100E051
S11358200921FFF7B0FE0346184610BD10B5012349
S1135830032900F18C0406D0062906D0072908D0D4
S1135840092913D016E00E2111E09AB11078002333
S113585007E0A178032906D062B1107820700023F4
S11358600320A07006E02246082100E00A21FFF789
S11358708AFE0346184610BD7B5F0000E95F000006
S1135880236000009160000037610000796100002E
S113589010B5044600F03AF900F027F851B1817CC4
S11358A08C4207D1002101604160817400F038F915
S11358B0002010BD00F034F9042010BD38B500F00C
S11358C017F800F012F819B1817C8C4200D113E072
S11358D007E038B500F00CF800F007F88C4200D16E
S11358E00AE000F01DF9042032BD614801687047E8
S11358F004460D4600F00AB9286000F011F90020B2
S113590032BD38B5FFF7F4FFFFF7EFFF21B1807C1C
S1135910844201D12960F0E7E3E7F8B50C46154667
S113592001261DB16946FFF7D4FF08B10420F2BD7A
S1135930002705E0491CC9B2032907D37F1CFFB225
S113594000984068017A8F421CDA002102680C2317
S113595013FB07230FF28412D3F808E09EF804E047
S113596002EB011C9CF80C207245E3D15868DCF86A
S113597008302A4621469847052804D00028DDD15E
S11359800026DBE73046F2BD70B582B00D46044612
S113599016466946FFF79DFF88B9012D08D1009985
S11359A0204600F06CFF009A02212046FFF7B5FF65
S11359B0009B5B685B68324629462046984776BD63
S11359C02DE9F843914601240F46B9F1000F18BFA1
S11359D0002F804601D0786808B9042045E000F023
S11359E095F8234E306828B1B17C884502D100F087
S11359F097F816E018B100F093F8022411E086F845
S1135A00128000F08DF8776032461A494046FFF75D
S1135A1009FE040007D03068FFF773FE4046FFF725
S1135A2037FF204621E000270FF2B00415E00025DF
S1135A30706800680C2111FB07012B01886800794C
S1135A401A19127B904203D11B590A1D40469847EC
S1135A506D1C032DECD37F1CFFB27068007A874263
S1135A60E5DB3068C9F800000020BDE8F2830000DF
S1135A700006FF1F8959000070B582B004466946CC
S1135A80FFF71CFF050027D1002517E0002600982A
S1135A90406800680C2111FB05000FF24001826888
S1135AA0127901EB06110B7B9A4202D140684968D6
S1135AB08847761C032EEAD36D1CEDB2009840682B
S1135AC0007A8542E2DB00980068FFF71AFE0500C1
S1135AD004BF2046FFF7DCFE284676BDA75400002D
S1135AE0F15400000153000001000000D5800000C3
S1135AF0C9810000E58100000300000000000000EF
S1135B000000000000000000000000000A480178C6
S1135B10002900D172B60178491C01707047000059
S1135B200548017800291FBF491E0170C9B2002928
S1135B3000D162B6704700001C09FF1F2DE9F04137
S1135B4004461D460E461746FFF7E0FF47EA46089F
S1135B5004EB081006F00F02C16A41F48043C362EB
S1135B6007F001016668760A760246EA42165B0A85
S1135B7046EA011603F0080333435D606368C06AB4
S1135B805B0A5B0243EA421242EA0111420A02F052
S1135B9008021143069A92054009920D00F0400054
S1135BA040EA024040F088000860FFF7B9FF00F0C7
S1135BB00CF9BDE8F08180B5C16A4A0A02F0080216
S1135BC012180C32026221F400610022826241F454
S1135BD0005108224262C16200920022036A00213D
S1135BE0FFF7ACFF01BD70B5011DFF224B6883F8C0
S1135BF088204B6893F8944044F0020483F894405E
S1135C0000234C6884F898300E68760A03F00F0479
S1135C10760246EA4416002500F038F846F00806F5
S1135C2000F034F846F0100635600E68760A760205
S1135C3046EA441444F01804256000EB431500249C
S1135C40EC6200255C0044F0010400EB0414E562FE
S1135C504C6804EB83045B1C082B84F8C050D3D33A
S1135C6000F5907005704B6893F8944004F0FD04BF
S1135C7083F894404B6883F88C2089224B6883F81E
S1135C8084204570486800F008F870BD35600E68DF
S1135C90760A760246EA4416704790F8941001F0AA
S1135CA0DF0180F89410704770B50C888B78C97840
S1135CB003F00F02DB09012943EA420505D1B4F5DB
S1135CC0806F0ED340F2FF340BE0412C28BF4024F8
S1135CD0816801EB820191F8C06046F0010681F809
S1135CE0C06000EB0511002BCD6A25F48045CD6220
S1135CF064F30905CD62CC6A24F40064CC6224F414
S1135D008064CC6214BF04210821846804EB8204FB
S1135D1094F8C050294384F8C01053EA020108BF24
S1135D20FFF749FF002070BD70B5044601F00F0570
S1135D30C80940EA4506204600F0FDF9A06800EBDA
S1135D408500002180F8C01004EB0610C16A890A9E
S1135D508902C162002070BD70B5044601F00F00D5
S1135D60C90941EA400204EB0212D36A23F48063B6
S1135D70D36223F40063D36200236668450145EAD5
S1135D800115760A45EA462503F0010645EAC605EB
S1135D902E68760705D5D66AB605B60946F0080614
S1135DA02E605B1C022BE8D3A26802EB800208433E
S1135DB092F8C03003F0FD0382F8C03004BF2046DF
S1135DC0FFF7F9FE00F001F870BDA06890F8941098
S1135DD001F0DF0180F89410002070472DE9F047AE
S1135DE0044684B0A06808228030017C0270C1F3AC
S1135DF003186068400A4002C1F3C00A40EA481030
S1135E00C1F3800140EA0A1040EAC1000068C0F30F
S1135E100949C0F383000D284AEA480004EB001541
S1135E200CBF01270027E86AC0F3803000284FD058
S1135E3004F5907007B1C170BAF1000F35D0A96AAA
S1135E404944A9626A6A561AE96A81F40061E962FE
S1135E5081F48051E96203D08905B9EB915F1CD2CA
S1135E60A96A0191296A0091E96A21F48041E962F1
S1135E708905B9EB915F08BFB8F1000F1BD1C07859
S1135E80696A04EBC000408A814214D2206800236E
S1135E9000220021FFF746FC1AE02A6A334648F044
S1135EA08001204600F0BDF812E059EA080111D142
S1135EB000200190009048EACA108DF808008DF87F
S1135EC0097069462068FFF7A0FBA068FFF7E5FEAC
S1135ED0BDE8FF87E96AC1F34033BBB963685B0A75
S1135EE05B02490A43EA481201F008011143496878
S1135EF02A6AAB6A9A18914206D0002302E05E5CDB
S1135F009E545B1C4B45FAD300210170A86A484497
S1135F10A862696A0E1AB8F1000F0DD167B1802129
S1135F20204600F008F9E06A40F40060E062E06BAB
S1135F3040F40060E06303E0E86A80F40060E86233
S1135F40E86A80F48050E862696A002918BF002E6C
S1135F5003D08005B9EB905F08D2A86A0190286A43
S1135F600090E86A20F48040E862A4E72A6A334695
S1135F704146204600F08CF8AAE770B515460FF2AA
S1135F80CC3282B0136800930C4630BB144E86F8B2
S1135F90220106F592710098F161B060FF2180F84A
S1135FA0801000220121304600F0E6F80D48B16867
S1135FB07060000A81F89C00B1687068000C81F878
S1135FC0B000B1687068000E81F8B4003046FFF785
S1135FD00AFE2E603460002076BD062076BD0000E7
S1135FE0B806FF1F0004FF1F08B90320704782682A
S1135FF0FF2182F88010816891F88420002281F8C2
S113600084200021826882F89810826882F89410B3
S1136010806890F8001141F0C00180F80011002060
S113602070472DE9F041804601F00F00400040F038
S1136030010008EB001782B0F86A1D460126C0F380
S1136040803030B9B8623A627D62F86A40F4005038
S1136050F86201F00F04F86A8005800DA84238BF89
S1136060054698F8210148B90095386AB96A0B18B1
S1136070012221464046FFF761FD0646B86A2843DF
S113608002BF002C4046FFF796FD3046BDE8F6817E
S11360902DE9F041044601F00F00400004EB001725
S11360A082B0F86A1E460125C0F3803010B9B86288
S11360B03A627E62F86A40F4005083059B0DF862F0
S11360C0B34238BF1E46BB6AD4F81CC09B18BCF14F
S11360D0000F04F5907211D092F800C0BCF1000FCB
S11360E00CD1412E0AD216F0030F08BF13F0030C93
S11360F004D020F40050F862E369157001F00F0831
S1136100507830B90096002241462046FFF716FD2C
S11361100546002E08BFB8F1000F09D1F86A80F4D3
S11361208050F86220F48040F8622046FFF743FD77
S11361302846BDE8F681E0B501F00F03CA0942EA3A
S1136140430200EB0212D36AC3F380338BB14FF0E6
S1136150FF330193136A8DF80810009300218DF822
S11361600910D16A21F48041D16269460068FFF7C1
S11361704CFA00200EBD0000F8B504460B4611464B
S113618001200CB90320F2BD0C2BFCD8DFE803F08E
S1136190072030363D676D70819D9D879A00A16808
S11361A0002081F80001A068017F490703D5017F21
S11361B041F080010177A06890F8081141F01001C6
S11361C080F80811A06890F8941041F0010143E0B0
S11361D0A068017F490703D5017F01F07F010177A2
S11361E0A06890F8081101F0EF0180F8081167E049
S11361F000296AD02046BDE8F44055E5002964D062
S11362002046BDE8F44009788EE500295DD00A787F
S11362101146204602F00F05D609FFF78CFF46EA27
S1136220450704EB0710C16A41F48061C1624A0A60
S11362306068400A400240EA451040EA061002F055
S1136240080289051043890941F08C010160A068A6
S113625090F8941001F0DF0180F8941030E0A1B3BD
S11362602046BDE8F440097876E571B3088027E05C
S113627059B30A7802F00F03082B26D2D00940EA5A
S1136280430004EB0010C06A800A00F0010048805B
S113629016E0D1B10878A16881F8980010E00025D3
S11362A045F08001C9B22046FFF73EFDE9B2204621
S11362B0FFF73AFD6D1C082DF2D32046FFF793FC3F
S11362C00020F2BD09B100200870F2BD00B970478A
S11362D03EB50468A06890F88050280744BF204663
S11362E0FFF77CFDE80712D5A168012084F821019D
S11362F081F8800069460020009010208DF8080085
S1136300002001908DF809002068FFF77EF9280627
S113631015D5A168802081F88000E06BC0F380204F
S1136320002802BFE06AC0F38020002807D0802143
S11363302046FFF711FD00212046FFF70DFDA06860
S113634090F85C1109B180F85C1137BD002007405A
S11363502DE9FC4104460F46904620681E4601AADA
S11363600621FFF73FFA9DF804000525012818BF10
S113637000282ED138781F21084208D1206804F162
S113638010020421FFF72EFA0546207C18E000F0E5
S11363901F01012902D10025258214E000F01F000D
S11363A0022812D1B8888DF800006A460020ADF8A2
S11363B0020005212068FFF715FA05469DF8020042
S11363C000F0030020820220306004F11000C8F8BD
S11363D000002846BDE8F68170B582B0054600206D
S11363E08DF800000C4628680DF101020621FFF724
S11363F0F9F99DF801000526012818BF002801D0ED
S1136400052076BD6078032804BF01208DF80000C4
S113641020781F21084208D1608801282BD12868E0
S11364206A461021FFF7B0FA24E000F01F000228AA
S113643004BF608800281ED1A0880F2108420ED115
S113644000F00F019DF8002041EAD0112868002ACD
S1136450C9B202D0FFF7ADF901E0FFF7B4F99DF836
S113646000102868002919BF221D0521221D0621BC
S1136470FFF753FA0646304676BD38B500F0B6F855
S11364809DF8000003280BD0012818BF022801D072
S1136490052032BD68888DF800006A4607210AE0AD
S11364A0206800220721FFF7C1F938B901208DF8CF
S11364B000006A4606212068FFF7B8F932BD2DE9CD
S11364C0FF470646904630680C469A4603AA0621C2
S11364D06788FFF787F99DF80C003D0A01284FF003
S11364E0050903D0010018BF02283AD1E0880190C1
S11364F0012D02D16A46092129E0022D04D18DF82B
S113650008706A460A2122E0032D07D18DF80A702B
S11365106A46A088ADF808000B2118E0212D05D1AA
S1136520A0888DF808006A460C2110E0222D05D1C0
S1136530A0888DF808006A460D2108E0232D0AD1B1
S11365408DF808706A46A0888DF809000E2130681D
S1136550FFF71AFA81460098C8F800000198CAF8B3
S11365600000484604B0BDE8F08770B5044682B028
S1136570154620681E466A460621FFF733F99DF842
S11365800000012818BF002801D0052076BD012095
S1136590306004F1100204F1100028601121206819
S11365A0FFF7F2F976BD38B500F020F89DF8000049
S11365B0012818BF002801D0052032BD002000F0BA
S11365C00EF8688810B9012000F009F82068AA1CA8
S11365D00321FFF7A2F92068AA1C07213AE08DF8ED
S11365E000006A4620680621FFF720B904460D46DC
S11365F020686A460621FFF7F5B8F8B500F043F8BD
S11366009DF8000008B10520F2BD0120386004F1B6
S1136610100204F1100030601221287920822068D1
S1136620FFF7B2F9F2BD38B5FFF7E0FF9DF80000BF
S113663008B1052032BDA888A97841EA002020824B
S113664004F1100220680421FFF767F9206804F1BF
S113665010020821FFF798F932BDF8B500F013F8DD
S11366609DF8000008B10520F2BDA888208204F13D
S1136670100220680821FFF7B5F804F11001316019
S113668002213960F2BD04460D46164620681F46B5
S11366906A460621FFF7A6B838B504460120052A44
S11366A00D460FD129786022114205D0090603D482
S11366B0E98809B103B90020C1012046BDE834408E
S11366C0FFF777B80598E9880268914238BF0160FE
S11366D003680498026800212046FFF723F858B99C
S11366E02978090608D5204601B0BDE830400023CA
S11366F000220021FFF71BB832BD2DE9F0418AB01A
S1136700044600200D4603900490052768689046CF
S113671010F1010F18BFB8F1000F10D002AA062122
S11367202046FFF75FF8287A0FF2B01C002808F122
S1136730080649D06868082801D1286808B90520E6
S113674076E04188718060258188B180C188F180BC
S113675042787270037833702B420AD15CF822506D
S113676028002DD004AB03AA31464046A84707466B
S113677026E0B9B1180615D4980602D500F072F8CF
S113678003E058061CD500F060F807000798049051
S11367900698039014D1F388039A00212046FEF74B
S11367A0C6FF45E0980602D500F05CF803E0580601
S11367B006D500F04AF80746079804900698039017
S11367C004A8019000232AE09DF80800032808D1BA
S11367D074785CF8244004AB03AA31464046A047D1
S11367E024E0686800281CBFF08800281FD0307897
S11367F001061CD4810606D500F01DF801212046AF
S1136800FFF78BF807E0400606D500F014F80F21D7
S11368102046FFF7B9F8074604A80190012303A80E
S113682000903A4631462046FFF736FF0746384681
S11368300AB0BDE8F08128680690059600208DF81E
S1136840200005AA68680790704700200690059606
S113685001208DF8200005AAF08807900F2120461A
S1136860FFF792B800200690059601208DF82000CD
S113687005AAF088079001212046FFF74EB830B5ED
S113688085B0044614480290039101208DF8040059
S113689002AA00208DF80300694680208DF80200CA
S11368A04020ADF800002046FEF74EFF050010D151
S11368B000208DF8020002AA69462046FEF744FF34
S11368C0050005D080212046FEF75BFF284600E046
S11368D0002005B030BD0000FB66000051630000DD
S11368E0D963000000000000D9630000000000002C
S11368F07B640000BF640000000000006B650000C2
S1136900A7650000FB650000276600005B660000C9
S11369100029817814BF41F0800101F07F0181706A
S1136920704700209AE0012098E040686549405C87
S113693070476449CA6842B18A6813780370501C6E
S11369408860C868401EC8607047002101707047A5
S11369505C49896908475A2806D15A4A01238B544D
S113696059495161916908477047FEB5554D044630
S1136970A9616068A2680221904766680FF2581006
S113698050F826706846FEF78CFA1020ADF8060021
S113699069464E488068006990F87900FF2818BF5E
S11369A0ADF806003846FEF731FA01213846FFF704
S11369B0AFFF40213846FEF70FFAFBF72EFB4FF4EA
S11369C07A71B0FBF1F04249B1FBF0F0002100E034
S11369D011464A1C00FB02F3322BF9D321B9B0F55E
S11369E0FA7F04D8012102E0202928BF1F21B879A9
S11369F000F0F0000843B87101213046FDF7DAFFDA
S1136A003448686101206168491908710020FEBD9D
S1136A1070B505462B4C686801190979A9B10FF2C4
S1136A20B80151F820600021FDF7C4FF0021304671
S1136A30FFF76EFF3046FEF725FA6868AA68002162
S1136A409047696809190020087170BD1D4881606C
S1136A50C260C1680029FCD10020704738B50546E2
S1136A600FF2740050F825402046FEF7C2F900F0FA
S1136A701201E17000F05001102911D04106114AB1
S1136A8014D54007A0780CD540F01000A070002069
S1136A908DF800006846116988479DF80000207150
S1136AA031BD00F0EF00A070207931BDA178C90696
S1136AB003D5C007EBD5A078F3E7207952692946BE
S1136AC0904731BDB400FF1F516900001000FF1F43
S1136AD040420F0057690000006006400070064005
S1136AE000600E4000700E407FB50646694674682B
S1136AF02046FBF7A3FB98BB0FF2481050F8245034
S1136B0001A8FEF79BFA009801902046FBF7A2FA31
S1136B10024601A92846FEF7E9F9F0B9B268022154
S1136B202046904701212046FDF75CFF4FF40011F9
S1136B302846FEF78EFAA86840F48020A860A8686A
S1136B4040F40020A8605A20384DA9688847A968F5
S1136B50A62088470120605503E02046FBF754FB3C
S1136B60002004B070BD10B50446304881606068F0
S1136B70A268012190476068FBF746FB002010BD26
S1136B8038B5044629486568285C48B10021284680
S1136B90FDF728FF0FF2AC0050F82500FEF72EFA9F
S1136BA02846FBF749FBA2682846BDE83840002187
S1136BB0104780B50FF28C03406853F82000FEF7AD
S1136BC061FA002002BD10B5194C00F01BF88002D8
S1136BD000D508E010BD10B5164C00F013F8800283
S1136BE000D500E010BD1149E0688968BDE8104097
S1136BF0C0B2084710B5104C00F004F8800200D56C
S1136C00F1E710BD2046FEF736BA10B50B4CFFF77E
S1136C10F9FF800200D5E6E710BD10B5084CFFF778
S1136C20F1FF800200D5DEE710BD0000880BFF1FD6
S1136C3000400C4000500C4000600C4000700C40C0
S1136C4000600D4000400C4000500C4000600C40BF
S1136C5000700C4000600D4010B50B46DFF8B444E2
S1136C60114601205B1E2268062B2ED8DFE803F0B4
S1136C70040A1519222D2C0039B30868400A00F0C3
S1136C80CAF804E009B30868400A00F08AF8E0B1E1
S1136C902268012182F8591410BDB1B158328A60BA
S1136CA010BD91B102F158008860BDE81040086839
S1136CB0400AB0E04FF40040086001224FF4007035
S1136CC048600A748860C860002010BD00207047C6
S1136CD070B5DFF840442060583000F070F9256842
S1136CE005F1580000F016FB06464FF4846105F1E7
S1136CF05400FAF767FF20680021C0F8606441651A
S1136D00002070BDDFF80C140860002009680865D5
S1136D10704738B5DFF8FC43206890F85C0430B95C
S1136D20FCF7E1FD2068012180F85C1441652068CE
S1136D3090F85D04A0B32168022081F85C0400F09F
S1136D40CBF80500F7D0206800F25C40C168002948
S1136D5004BF0178022903D1032000F0E6F801E022
S1136D600121417042F27D70854219D0206800F201
S1136D705D400021017042F274718D4202D1022102
S1136D80C17431BD42F212718D4203D10221C1742A
S1136D90032002E00321C1740020BDE83240C4E0B6
S1136DA031BD70B50446B4F5847F82B00D4630D34E
S1136DB0D84E306800F25B410A7862B9887808B12D
S1136DC00F2076BDA868694600F074F808B30098EF
S1136DD000F097F803E0D0F86404844219D13068D5
S1136DE06A6800F264414B68934238BF1A468E6861
S1136DF096199B1A641C8E604B600C6013B90021B9
S1136E0080F85B1400F51670A968FAF7DFFEFFF747
S1136E1080FF002076BD38B50C4605466168A06841
S1136E20FDF756FD0FF2984000E00C30416831B197
S1136E300268AA42F9D18268A068FAF7C7FE0FF285
S1136E40043045B140F201116D1A0DD06D1F19D0F7
S1136E506D1E1BD027E0A168552081F8FE01AA20F1
S1136E60A16881F8FF011EE0A16801F5BE7400F07D
S1136E701CF80A682260097C50F8210000F04AFAE4
S1136E80206210E0A06800F09AF80CE000F00DF821
S1136E90097C50F82150284600F03CFA0246A068CC
S1136EA02946FAF793FE002032BD9A49096801F594
S1136EB08C6170474269984B9A4202BF426B974B70
S1136EC09A4204BF027E012A04D1C069000108600D
S1136ED001207047002070478E480068D0F86C2469
S1136EE0B2F5007F04D2110004D142F27D707047E4
S1136EF04FF40071521AC0F86C2400F51670FCF7B8
S1136F0034BD8449096801F25A4201231370537055
S1136F1001F58D61002393700123D3700023137155
S1136F2008604B600120087270477A49096801F2D1
S1136F305A42012313709070002301F58D60537041
S1136F40D37013710121436003600172704730B53F
S1136F503022027078224270002282720FF2D01323
S1136F609400C4F11C0421FA04F505F00F0415186B
S1136F70E45CAC70521C082AF2D330BD10B5002278
S1136F8061B10A23B1FBF3F30A2404FB131130317A
S1136F901154521C19460029F3D102E0302101702A
S1136FA00122002111541118491E05E00A780378C2
S1136FB001F8013900F8012B8842F7D310BD70B5F0
S1136FC004465748C0B080680569286814904FF695
S1136FD0FF70B5F87A608642524808BF41F288369D
S1136FE0016826A8FFF7B3FF55F8101F0DF1A300A1
S1136FF0FFF7ADFF286869680818411E0DF1AE005F
S1137000FFF7A5FF69690DF1B900FFF7A0FF6869F3
S1137010A9690818411E31A8FFF799FFA96C0DF161
S1137020CF00FFF794FFE96C0DF1DA00FFF78FFF53
S1137030296D0DF1E500FFF78AFF696D3CA8FFF7A4
S113704086FF696815A8FFF799FFA9680DF15F002D
S1137050FFF794FF29690DF16A00FFF78FFFA96913
S11370600DF17500FFF78AFF314620A8FFF786FF70
S11370702D4801680DF18B00FFF780FFAA6D2B4BA3
S113708022A023A19A420CBF0A4602462B6A03B1EE
S113709008460F900DF18B033CA80E9013930DF14D
S11370A0E5000D9020AB0DF1DA000C9012930DF178
S11370B0CF000B90119231A80A9010910DF1B900F4
S11370C009900DF1750008900DF16A0007900DF11B
S11370D05F0006900DF1AE0005900DF1A300049041
S11370E015A8039026A802909DF850009DF85230F0
S11370F09DF853200FF25C0101909DF8510000901F
S1137100204600F023F940B070BD00006E6F00000F
S1137110796573009C0BFF1F53544D507367746C57
S11371201000FF1F248004406001FF1F6B6366672B
S113713030313233343536373839616263646566E9
S113714000000000E4060000EC060000FC0600005D
S1137150080700004B696E6574697320426F6F7491
S11371606C6F6164657220256325642E25642E2569
S1137170640D0A0D0A53797374656D20646576692C
S113718063652049443A2025730D0A466C6173688F
S11371902073697A653A2025732062797465730DCA
S11371A00A466C6173682072616E67653A202573C4
S11371B02D25730D0A466C61736820736563746FC3
S11371C0722073697A653A20257320627974657335
S11371D00D0A466C61736820626C6F636B733A20AE
S11371E025730D0A52414D2073697A653A2025733F
S11371F02062797465730D0A52414D2072616E6785
S1137200653A2025732D25730D0A526573657276D0
S1137210656420726567696F6E20303A2025732D8E
S113722025730D0A5265736572766564207265670D
S1137230696F6E20313A2025732D25730D0A56652A
S113724072696679207772697465733A2025730DC3
S11372500A436865636B20726573657276656420A2
S1137260726567696F6E733A2025730D0A426F6FFA
S11372707420636F6E6669672070726573656E74DF
S11372803A2025730D0A5065726970686572616CE5
S113729020646574656374696F6E2074696D656FCD
S11372A075743A202573206D730D0A43505520637D
S11372B06C6F636B3A20257320487A0D0A00000036
S11372C00000000014070000360000000100000068
S11372D04C0700000E000000010100005C070000E4
S11372E0A001000003010000FC0800006000000091
S11372F004010000AC090000A0000000050100002A
S11373005C0900004D0000000000000000000000C7
S11373100000000000F10103810704D010F8011BF4
S113732089B18107FAD10268B2F10131914311F0B8
S1137330803F04BF50F8042FF6E710F8011B11B189
S113734010F8011BFBE7C01A704700000CB41CB511
S1137350044604A801900A46009401AB6946074814
S11373607844183000F018F8009A002111700028B1
S11373705CBF0098001B16BC5DF80CFB2B9AFFFF4A
S113738070B504461E000846154604D015F8011BC6
S1137390A047761EFAD170BD2DE9F04784B082462D
S11373A0894614461F46E84607E00123224649461B
S11373B05046FFF7E5FF8146641C207810B904B0FD
S11373C0BDE8F0872528F0D16078A41C2528014663
S11373D018D058285CD063280ED0642818BF6928B8
S11373E014D06F2854D0702858D073285DD07528D5
S11373F018BF78284CD0E0E73868386050F8041B90
S11374003860C9B24846D0478146D6E73868386004
S113741050F8045B3860002D03D52D214846D04731
S1137420814664206F2808BF082205D040F020015F
S1137430782914BF0A2210220B216428AC4603D1F8
S1137440002D48BFCCF1000CBCFBF2F502FB15CCBF
S11374500CF130065FFA86FC4B1EBCF13A0FA4BF58
S1137460A0F15106B44403F808C019465FEA050CBC
S113747001D00129E8DA68460D184846D1F10B0914
S1137480C2D015F8011BD047B9F10109F9D1BBE706
S11374903968396051F8045B3960C3E7386838608B
S11374A050F8045B38607820BCE73868386050F8DE
S11374B0045B38602846FFF72DFF06004846A3D03A
S11374C015F8011BD047761EFAD19DE710B5C248C6
S11374D08068006900F1680434214AF2C030F9F789
S11374E0DAFC48B934224AF2C0312046FAF77EFB6E
S11374F02068BA49884204D0FF2234212046FAF792
S113750065FEFAF7BDFD002010BD38B5B24DA86880
S113751004694B20E07004F110020220A0700421E1
S11375200020607020705020E0710120A0710220C2
S11375306071002020715420E0720120A0720020AC
S11375406072207201202063A548606305F1200069
S11375502B69DB6A98472B69DB6A04F11402012169
S113756000F066F82B69DB6A04F11802002100F0D0
S11375705FF82B69DB6A04F11C02022100F058F861
S11375802B69DB6A04F12002032100F051F82B6916
S1137590DB6A04F14402052100F04AF82B69DB6A36
S11375A004F14802062100F043F82B69DB6A04F178
S11375B04C02072100F03CF8A0698A4A404252423A
S11375C04FF0FF310240891A874AE1651040A065F7
S11375D0002186482066864860666869E16007E0A5
S11375E094F87830134202D0E3681A43E260491CED
S11375F0182202FB01021268002AF1D17D480168B9
S113760021644168E1638068A063686850F8101FD2
S1137610616241680068081A401CA0622046FAF7BB
S113762049FF01202065F9F72CFC6065002032BD7C
S113763005F12000184700002DE9F8431546664A75
S11376406D4C884691680427401E0E691928994696
S11376505FD8DFE800F00D17191B1D1F25275E29D1
S11376602B325E212335384447494B4D4F51535CEF
S1137670B9F1000F18BFC9F8007005B12E600020E1
S1137680BDE8F2830C36F3E71036F1E71436EFE782
S11376901836EDE72036EBE72436E9E72836E7E746
S11376A03436E5E72C36E3E73036E1E7D069416963
S11376B04969884720602646DAE710275836D7E715
S11376C04E480068F6E702F12000126992696946A3
S11376D090479DF800000028ECD00120EAE70C2731
S11376E03836C5E74436C3E74836C1E74C36BFE70A
S11376F05036BDE75436BBE70836B9E79C36314609
S1137700404600F031F80028BAD11827B0E7B43663
S1137710AEE742F63C00B3E72F4A92681369401E75
S1137720072842F63E0219D909380BD0401E012819
S113773084BFC01E032811D9083809D0401E03286D
S11377400CD90EE0002918BF012903D11963704731
S1137750032901D3104670471965704742F63D006E
S1137760704742F63C007047F0B589B00C46244D92
S113777000E008352DB1696800291CBF29688142E1
S1137780F7D16A68100008BF042023D0694600209E
S113779090470098F0B903AE0290012700200190B1
S11377A001A96A683846904740B9019830600121C0
S11377B002987A1E91400843029001E00020306054
S11377C0361D7F1C062FE9D3182202A92046FAF79A
S11377D00DFA002009B0F0BD1000FF1F6B6366674F
S11377E0FFEF030004930000000000000000FF1FEF
S11377F04F28FF1F588004406C0CFF1F2480044056
S113780074060000AF49D1F88820531C5218C1F8FF
S1137810883082F82000D1F8880000F03F00C1F8D9
S11378208800704700207047B8E02DE9FC410C0047
S1137830154614BF002D0420984628D0A14F0020DF
S113784007F190062860707000F0A8F818B11EE0E7
S1137850A22000F075F820213846FAF7B3F9424621
S11378603946684600F0F8F810B1002129600EE0AE
S11378703946684600F042F9BDF804108142E7D168
S1137880012030702760BDF8020028600020BDE8A8
S1137890F6812DE9F0410C0082B015461E4635D024
S11378A0212D33D200F07AF800283FD1DFF814827A
S11378B098F8910010B1002088F8910008F1600751
S11378C05A203870A42078700EB1A52078707D807D
S11378D02DB12A46214608F16600FAF777F908F136
S11378E06601384600F00AF9B880A91D384600F050
S11378F064F8D8B9684600F0EFF8B8B99DF801000B
S1137900A12812D0A22806D0A32801D004200DE07B
S113791042F212700AE07888811D384600F04DF872
S113792020B99DF80100A228E4D00020BDE8F6812A
S11379306548012181700021017070472020704743
S113794080B55A218DF800108DF8010001205D49A1
S113795081F891000221684600F02FF802BD10B5AD
S11379600446594882B00178427880781140014237
S113797011D10FF2B8100088ADF80000022223697B
S11379805B6869462046984723690FF2A4115B6837
S113799008222046984742F2137016BD4A480178DF
S11379A019B100210170A12004E0817819B10021EE
S11379B08170A320C4E700207047444AD3690A4673
S11379C0014618461B695B6818472DE9F14F8B4641
S11379D01646FAF765F904464FF47A708846704300
S11379E0FAF768F9DFF8DCA00027064689460AF1B1
S11379F088050EE06868296888420CD050440099D4
S1137A0090F8200078547F1C6868401C00F03F0008
S1137A1068605F451DD0FAF743F9021B61EB080368
S1137A2041450AD828BFA04207D2E2436FEA0803BF
S1137A3010185941421C41F10003B9F1000F08BF6D
S1137A40002ED7D04B45D5D301D8B242D2D305208E
S1137A5000E00020BDE8F28F70B582B005460C4608
S1137A60164600F039F858BB6878A62804D11748A0
S1137A70C069FFF774FF76BDA42106B1A521884231
S1137A8001D0012076BD00F023F8BDF80010698014
S1137A90B0B908462128A8BF2020688000F018F853
S1137AA0BDF80010A98058B9698849B12046FCF78F
S1137AB00FFF69880A2000FB01F22046FFF785FFCB
S1137AC076BD00003013FF1FC013FF1F1000FF1FFF
S1137AD014220221684678E710B5044600220121E9
S1137AE02046FFF772FF40B920785A28F6D1601C6F
S1137AF0BDE810400A22012167E710BD30B583B00C
S1137B0004460D466846FCF787FF04222146684672
S1137B10FCF785FF628829466846FCF780FF01A9C7
S1137B206846FCF7A8FFBDF804003EBD5AA7000054
S1137B30000201500000AAEA05484CF22051C1811C
S1137B404DF62811C1814FF4E9710180704700BFDF
S1137B500020054005207047087A18B918480860C5
S1137B604C2006E005207047052070471548086042
S1137B701220486000207047087A18B9124808603B
S1137B804020F6E70520704710B5887A0F4A10B9EF
S1137B90136850680FE092680B891489A34202D1DC
S1137BA0042800DA01D1052010BD1368526853F887
S1137BB0203052F8200048600B60002010BD000007
S1137BC0CC01FF1F1802FF1F2C02FF1F7003FF1FB1
S1137BD0002101604160FB3041700170002070475A
S1137BE010B5044604F15800811C00220A708A7200
S1137BF0CA7204F130010A6840F8142F0A79D209D4
S1137C004275C87998B303282CD004283ED0122892
S1137C101ED0152849D01A2842D01B2859D01D2817
S1137C204DD01E282DD0232844D0252833D02828F1
S1137C3013D02A2820D02F2846D0552835D05A28AA
S1137C402ED09E2827D0A82807D0AA2814D045E0F3
S1137C502046BDE8104000F03CBD2046BDE8104081
S1137C6000F049BD2046BDE8104000F027BD204685
S1137C70BDE8104000F08ABD2046BDE8104000F089
S1137C804ABD2046BDE8104000F06ABE2046BDE86B
S1137C90104000F040BE2046BDE8104000F0C3BDD7
S1137CA02046BDE8104000F07EBD2046BDE81040EF
S1137CB000F093BD2046BDE8104000F0C9BD204649
S1137CC0BDE8104000F072BE2046BDE8104000F050
S1137CD05EBD2046BDE8104000F069BE204600F0BD
S1137CE08CFE04F1EC0100220A704A70CA708A709A
S1137CF00A72CA7110BD2DE9F0410C4684B01546D4
S1137D0062682F1D12F1010F4FF00108284605F19A
S1137D10ED0618D1317800291EBF39680968002999
S1137D2065D095F83710282918BFA8295FD10021FC
S1137D3001916A46216802910021009101213B686A
S1137D401B68984753E0BB68934224BF9A1ABA60F1
S1137D50B279012A09D10020B07186F8018030700F
S1137D60317B2868FDF725FD41E03278002A02BF07
S1137D7062680D2A2168327852B33968096800298B
S1137D8035D06168019121680291F968009195F8F4
S1137D903710282918BFA82904D13B681B686A46F4
S1137DA001219847B86848B1F86861680818F86014
S1137DB0284600F01AFB8046B868C0B9002030702D
S1137DC00D23317B286805F14802FDF7ABFC0EE07A
S1137DD060680D2802BF0868DFF8D813884206D10E
S1137DE086F80380717B00F0FAFA86F80880404632
S1137DF0D0E02DE9F0410C4684B09046626800263C
S1137E0012F1010F08F1340108F1EC07404608F1C2
S1137E10040515D17A78002A1EBF2A681268002A40
S1137E200DD0C9782A2918BFAA2908D101966A4613
S1137E3021680096029102212B681B689847A8E0EC
S1137E40AB68934224BF9A1AAA603A7A012A07D1EE
S1137E500120F8703E723E707E7200F09EF898E049
S1137E603A780AB36268019222680292EA68009240
S1137E702A6813681A0011D0C9782A2918BFAA29B8
S1137E8002D16A4602219847A86850B1E86861683F
S1137E900818E860404600F0D7FA0646A8680028AB
S1137EA077D1002038705EE03879002866D06068A9
S1137EB01F2802BF686AC04A90425FD14A78F02006
S1137EC0024202BF8B78E024234257D1387B401C06
S1137ED0824253DA002B51D0112B4FDA7E72AE60FE
S1137EE0CE61B4484861A86A88613E71E86AE86274
S1137EF00A78120602D410B1012000E00020387084
S1137F000878000603D5E86A10B1012000E00020DB
S1137F107870787800281EBFB8780028012039D1FD
S1137F204046FFF75DFE0646052E14D13878012839
S1137F3006D1F87808B9012038720020387008E0BA
S1137F407878012805D1B87808B90120F8710020A3
S1137F5078700220F8723878002804BF78780028F6
S1137F6017D1F879A8B9797BD8F800000D2308F166
S1137F704802FDF7D7FB0120B8720AE000F00DF8C3
S1137F80797B00F00BF801203E71F870B870F8723C
S1137F907871304604B0BDE8F081B97BD8F80000B0
S1137FA0FDF707BC2DE9FF47044604F1EC066068C1
S1137FB08068317C427900258A424FF0010A22D33D
S1137FC0006800B300EBC1000838002100E0491C40
S1137FD00278914217DA42680C2303FB01221378DA
S1137FE0082BF4D196F80FC0002000E0401C117A51
S1137FF0884205DA516803015F5C6745F6D15D1874
S1138000D07870740DB901204EE0A5604FF00009DE
S11380106A4FDFF8AC8108E0039402AA206869463D
S1138020FDF792FB824609F10109287981451CDAA2
S113803000208DF80400A86810F829008DF80200CB
S1138040A96801EB89014988ADF80010A96801EB22
S1138050890149788DF80310C109012907BF70739C
S1138060CDF80880B0730297D6E7002030707070A6
S1138070F070B0703072F071012030710020E06057
S11380807071B071F072707A012803D1B17B2068ED
S1138090FDF750FBB17B20681F2304F12802FDF794
S11380A046FB01207072504604B0BDE8F08738B535
S11380B004460120A16861B1002506E0886810F833
S11380C025102068FDF75DFB6D1CA1680A799542B7
S11380D0F4DB32BD2DE9F0413A4D86B00F462968F4
S11380E0144609B1022062E02946FDF70AFC0600A5
S11380F004D02846FFF76CFD304658E0286820B9C4
S11381002846FFF765FD032051E06F60002005F16C
S1138110F507F871FF206B68B8712E461B686A4634
S11381200521304698478046019800281CBF0099D5
S1138130002938D09DF81010009AF9706A61491E20
S1138140F970702202992962A86103996962002179
S1138150E96105F158010A700A22CA7100228A7085
S11381608A816A69521E02F47F431B02150A43EA9C
S1138170026305F47F452B43050A05F47F4543EA72
S1138180126200F47F431B0243EA00632B4343EA79
S113819010600863C863CA6200208A63387078700C
S11381A02660404603E02846FFF712FD012006B092
S11381B0BDE8F0815553425355534243F37D0000CB
S11381C0F77C00001C08FF1F38B5040001D1032010
S11381D032BDFFF76CFF05462046FFF7F9FC284641
S11381E032BD00002DE9F8430546160014BF002DEA
S11381F003204FF0010800F0EA802C1D491E0529D8
S113820005F1EE0706D8DFE801F0A80306162D50A5
S11382100020B873DAE0206800281EBFB87B3178EC
S11382208142F7D010B12846FFF741FF3078B87388
S11382300020787311E020680028EBD03088F97BA7
S113824006460004B1EB106F0BD1787BF6B2864280
S113825007D02846FFF72BFF7E732846FFF7A2FEC0
S11382608046B3E0206800281CBF60680028F8D06E
S11382704FF00009606801798945F2DA00F0A9F845
S113828010D1387828B92868FDF793FA8046012080
S11382903870787830B931782868FDF78AFA8046E2
S11382A00020387009F10109E4E7206800281FBFA5
S11382B060680028F8780128D3D04FF0000917E04F
S11382C000F087F812D13878012805D12868FDF725
S11382D07AFA8046002038707878012806D13178FF
S11382E02868FDF770FA80460020387009F101090A
S11382F0606801798945E3DB787A032818BF02288E
S113830013D13879012813D0387A012803D1F97AA6
S11383102868FDF70FFAF97A28680D2305F1480259
S1138320FDF700FA002038727872387901284DD1AF
S11383303878002804BF7878002847D13871387A13
S1138340012803D1F97A2868FDF7F4F9397B00F0A4
S113835046F800203872787238E03168087800F006
S11383601F02012A01BFFA7B8B88DCB294422DD113
S11383704C78FE2C02D0FF2C11D027E0934204BF8E
S11383804A88002A20D1C98802291DDA00061BD593
S113839005F1F80070603068C088B06016E0934260
S11383A004BF4A88002A0FD1C98869B900060BD4D2
S11383B02846FFF77CFE2846FFF7F4FD80460020A0
S11383C0F8700120387101E04FF005084046BDE81F
S11383D0F2838068317810F8290081427047286858
S11383E01F2305F12802FDF7A2B93EB500F061F89C
S11383F0206AB0F1011F28BF4FF480300190019929
S1138400E068814238BF0846029501900421636800
S11384101B682046984700F046F804F1ED0007D2A7
S1138420017B019B029A2068FDF77CF9054609E06F
S1138430012141708571022181720570017B2068E0
S1138440FDF7B7F928463EBD3EB500F032F8606A44
S1138450B0F1011F28BF4FF4803001900199E0680A
S1138460814238BF084602950190032163681B6866
S11384702046984700F017F804F1EC0007D2817BFE
S1138480019B029A2068FDF752F9054609E0012193
S1138490C17005720221C1720570817B2068FDF7ED
S11384A088F928463EBD6269A36921695A4391420D
S11384B0704704460025206900906A46704710B54D
S11384C0536884696343C360126883695A430261D1
S11384D0012904BFBDE81040FFF787BFBDE8104085
S11384E0B2E700002DE9F041044604F16C050020D8
S11384F0296804F1580829B921656968002900D060
S113850002219CE0687D0028686808F1020704F1F4
S1138510EF0640D020B9216500F0CAF878B961E0CF
S1138520AA7D002A2ED088420DD200F09CF802D1F8
S113853000F093F801E000F0BBF8002852D000F0FE
S113854086F8112053E0814209D100F092F802D15B
S113855000F083F801E000F0ABF860B96EE000F0E1
S11385608EF804D100F098F800F079F801E000F0FA
S1138570A0F800285CD0012184F85410032139703C
S1138580112161E02165AA68B17A20680023FDF712
S1138590C9F8022026E048B9F17A2068FDF709F904
S11385A028682065012084F854000BE0AA7D5AB1A4
S11385B0F17A2068FDF7FDF828682065022084F828
S11385C054000120307013E0884213D200F04BF8BD
S11385D005D105F10C02002100F042F801E000F0A1
S11385E055F810B984F8540002E000F030F8B8727D
S11385F005202AE081420FD100F03BF805D105F1B6
S11386000C02002100F02CF801E000F03FF8A8B1C2
S1138610012184F8541015E000F031F805D100F080
S11386203BF8002100F01CF801E000F030F848B9F4
S113863098F82810012908BF022100D0002184F8ED
S1138640541002E003213970B972BDE8F0810120B1
S113865084F8540003203870704705F10C0201219E
S11386602046FFF72CBF081A206598F82800012837
S113867070470020206598F82800012870470020E2
S1138680206598F828002B68012870476B68AA6851
S1138690F17A2068FDF74BB8A0692968B3FBF0F0C4
S11386A02861A26902FB1010206505F10C027047D5
S11386B06B68AA68B17A2068FDF734B800F15801F4
S11386C001F11802122313605160012300219374F5
S11386D0BCE038B500F1580101F1400200230FF26B
S11386E03C341D5D9D545B1C242BFAD301F118020C
S11386F04031242368E070B500F029F8282E04D115
S113870059799B7943EA012102E0A82E00F032F85E
S1138710183201230EE070B500F019F82A2E04D1A6
S113872059799B7943EA012102E0AA2E00F022F84C
S11387301832002393742B6894604B431360D16008
S11387400023536001231374BDE87040CAE600F1AE
S1138750390300215D781C782D0445EA04649D7872
S113876044EA0524DD782C4300F1180500F1580291
S1138770EE7F704709D15E791979360446EA0161C2
S11387809E79DB7941EA06211943704700E000BF76
S113879000F15801002241F8182F01228A740022A6
S11387A04A600A749EE638B500F1580101F164028A
S11387B000230FF28C241D5D9D545B1C082BFAD3FF
S11387C001F1180264310823516013600021012370
S11387D011749374BDE8324084E638B5044604F15C
S11387E0580505F1640000210FF254228B5C0B54F0
S11387F0491C0829FAD305F1180008210160012158
S1138800817405F164014160002101742046FFF781
S113881069FE94F83810C90704D5A91C05220A700A
S113882024228A7232BD90F8373000F15801252B8A
S113883001F1180203D1082313602C3102E00C2348
S1138840136034315160012191740021117449E69F
S11388502DE9F0410FF2C01186B00968009100F1D2
S1138860580890F83F5098F86C60002100220023CB
S113887000F1140426B1A668002E14BF02260326B4
S113888027680197D4F804E00397F400F7000C3745
S1138890CDF808E08DF80340CDF810E0BD4288BF64
S11388A03D466F46D2B201EB0804D75D521C491C09
S11388B0042984F86D70F4D3002203AFC9B2D75DE4
S11388C001EB0804521C491C082A84F86D70F4D387
S11388D098F86C208AB100220CE001AFDBB201EB06
S11388E00804DF5D84F86D705B1C491CC9B208295B
S11388F0F3D3521CD2B2B242F8DB012208F11801C0
S11389008A7408F16D024A600D6000220A7406B090
S1138910BDE8F041E6E538B5054605F1580404F133
S1138920180000210160012181740021416001745B
S11389302846FFF7D7FD05F138010A7F022A0ED039
S11389400A7802F01F02172A02D100220A7732BDE8
S113895001220A77A11C05220A7024228A7232BDE0
S11389602DE9F041044604F13B0604F1580537783B
S113897005F118000021016000F038F88046707E8F
S1138980022808D0F80706D5012070760521A81C16
S113899001702421817260680368180003D00022EA
S11389A00721204698474046BDE8F081F0E670B5BF
S11389B082B0044604F13B0504F15800297801F023
S11389C003018DF80010002140F8181F00F00EF884
S11389D00646687E022807D060680368180003D042
S11389E06A46082120469847304676BD01218174A5
S11389F0002141600174204674E500F15801002211
S1138A0040F8502F0122027105208870202008733D
S1138A10002048737047000000000000008004023A
S1138A202000000046534C2053454D4946534C20EA
S1138A304D4153532053544F524147453030303108
S1138A400000000000000000DFF8D8130A7B01F2E8
S1138A505A4100200B7803B10120DFF8CC331A709F
S1138A605870C97F002914BF1043002070470000CC
S1138A7070B50024491E1546DFF8A833112903F107
S1138A80080603F279425CD8DFE801F0095B5B5B1E
S1138A905B5B0B1A3D42474C51565B5B292E1470AD
S1138AA04FE0002D4DD001201070287850702978A7
S1138AB03068FCF762FB2978B06CFEF707F940E0F8
S1138AC0107800283DD02A88110A022939DAC818FA
S1138AD080F87B24D2B23068FCF763FB31E0002DD0
S1138AE02FD0507828702CE05DB32A88100A022811
S1138AF007DAC01802F47F4190F87B040843288009
S1138B001FE005241DE0E5B12946FFF72FF817E023
S1138B10BDB12946FFF730F812E095B12946FFF7B9
S1138B2033F80DE06DB12946FFF714F808E045B1BC
S1138B302946FFF711F803E01DB12946FFF714F8A1
S1138B400446204670BDF8B50FF21030B54C0078DD
S1138B50B64E8DF8000005464FF490612046F9F7B3
S1138B6031F8F9F741FA0028B06800690CD190F89F
S1138B70781001F0EF0180F87810B0680069C168DE
S1138B8021F01001C1602DE000F17C064FF6FF7169
S1138B90728830888A4208BF884209D0A449087282
S1138BA03088000A4872708888727088000AC87217
S1138BB07068A04F10F1010F04D01021F8F76BF981
S1138BC000B977689C489D4E076004F58F600021CA
S1138BD001800020A0602065206022463146FCF719
S1138BE0EFFE08B10120F2BD30680069206520461F
S1138BF0FEF76EF830684068A0602046FCF7DFFAA4
S1138C0068B2010007D58E4A01F00F039A1840207C
S1138C1002F8040C02E08B4B4022C254012005F000
S1138C201F029040884A490942F821002068FCF755
S1138C3065FD0020F2BD10B50020FCF71DFFA0B9B2
S1138C40784C2046FEF75EF82046FCF7BCFA7F48D5
S1138C500168490309D57E4A4FF4001111607D4A29
S1138C601160016821F48021016010BD38B56E4C9B
S1138C70794D0020207001206070F9F796FAFEF714
S1138C8048F8A878032803D10020A870FAF7A2FEB8
S1138C90F9F791FA287800B1012060700120207062
S1138CA031BD10B55F4C002104F11400F9F762FAEC
S1138CB0002104F11800F9F75DFA04F11400F9F742
S1138CC065FA002010BD2DE9F0410C00154614BFD3
S1138CD0002D042039D00020286013B1012B02D0CC
S1138CE02CE0012600E002264F48007860B3DFF84C
S1138CF0348108F10807B87930B13868242308F1C1
S1138D0020020221FCF711FC0120B8714FF0FF3161
S1138D1008F11400F9F730FA387EB04206D0012E7B
S1138D2008BF02280AD142F212700EE0B87EF97E22
S1138D3040EA01207969091F814201D2012004E03F
S1138D4008F12401216028600020BDE8F0812DE9AC
S1138D50F0413548007800280C4615463ED0212DB8
S1138D6028BF04203BD213B1012B10D011E00327FC
S1138D70DFF8B080F9F719FA08F10806707950B1F4
S1138D8000207071F9F717FA42F2127027E00427F5
S1138D90EEE7012023E0F9F70EFA3776002070762B
S1138DA0B576280AF076002C18BF002D05D02A4687
S1138DB0214608F12400F8F709FF98F84600012835
S1138DC00CD13068242308F120020121FCF79DFB1B
S1138DD04FF0FF3108F11800F9F7CEF90020BDE893
S1138DE0F08110B54469A468002300220021A04743
S1138DF010BD002070472020704710B5094C94F82E
S1138E005C04022818BF032807D104F11400F9F701
S1138E10C1F904F11800F9F7BDF92068BDE8104064
S1138E20FDF754BAC813FF1F4818FF1F1000FF1F97
S1138E301802FF1F7003FF1FC413FF1F8C00FF1FC6
S1138E4018ED00E000E400E000E100E034800440BC
S1138E5084E100E084E200E02218FF1F35000000F6
S1138E6000F00BF8002801D000F00AF80020C046FA
S1138E70C046FAF769FFFAF783FF01207047000044
S1138E8010B5074979441831064C7C44163404E083
S1138E900A68081D511888470146A142F8D110BD3F
S1138EA04C04000060040000C3250000D12500002C
S1138EB0EC0400008009FF1FCC060000D000FF1F57
S1138EC0DC0A00000000FF1F7C050000640A0000AB
S1138ED0D4050000000000000000000000000000B5
S1138EE0000000000000000000000000000000007E
S1138EF0000000000000000000000000000000006E
S1138F00000000000000000000000000000000005D
S1138F10B809FF1FF809FF1F95010000C9500000A0
S1138F20000000009801FF1F596C000000000000C1
S1138F30C401FF1F7400FF1F718A000002000000BB
S1138F40000000000000000000000000000000001D
S1138F50994A0000B74A0000000000000000000029
S1138F600000000000000000000000003369000061
S1138F70576900000000000000000000FFFF03002C
S1138F8001000000840600000000FF1FFFFF022014
S1138F90010000004C0A000000000068FFFFFF6FA2
S1138FA000000000F00A000000000004FFFFFF07BB
S1138FB000000000080B000000000040FFFF074015
S1138FC0000000004406000000000840FFEF0F40CE
S1138FD0000000004406000000F00F40FFFF0F40B7
S1138FE00000000044060000000000E0FFFF0FE066
S1138FF00000000044060000000000000000000023
S11390000000000000000000000040018103400057
S113901002034000830240000402400000000000FC
S1139020020000006401FF1F0000000003000000B4
S11390307401FF1F01000000010000008401FF1FF4
S11390409001FF1F01010000000000000200000069
S11390506C01FF1F0000000008065001A001FF1F63
S11390600100000001000000B001FF1FBC01FF1F50
S1139070030100000600FF0901A10185011901296E
S113908001150026FF007508952391028502190138
S11390902901150026FF00750895239102850319FF
S11390A0012901150026FF00750895238102850416
S11390B019012901150026FF00750895238102C0B6
S11390C01201000200000040A21573000200010218
S11390D00301000009024000020100C0320904003B
S11390E0000203000003092100010001224C0007D3
S11390F00581034000010705020340000109040142
S11391000002080650030705830240000007050417
S113911002400000040309043A03460052004500DB
S113912045005300430041004C004500200053001B
S113913045004D00490043004F004E0044005500D7
S1139140430054004F005200200049004E004300E9
S11391502E0000002A035500530042002000430063
S11391604F004D0050004F0053004900540045008B
S1139170200044004500560049004300450000001B
S11391803E034D004300550020004D0053004300B2
S1139190200041004E0044002000480049004400E3
S11391A02000470045004E0045005200490043009E
S11391B020004400450056004900430045000000DB
S11391C02203420041004400200053005400520096
S11391D049004E00470000000000000000000000AD
S11391E000000000040000003A0000002A00000013
S11391F03E000000220000006C02FF1F7002FF1FEF
S1139200AC02FF1FD802FF1F1803FF1F5003FF1FEC
S11392103C03FF1F090400006C02FF1F0400000050
S11392206403FF1F01000000F7F7F2B830B504E053
S113923012F8014B00F8014B491ED1B1C507F7D410
S11392400129F5D0850701D4042904D232F8024B50
S113925020F8024B891E8B08EFD000EB830403E057
S113926052F8045B40F8045BA042F9D3A1EB8301FC
S1139270E3E730BD80B513460246184600E080B5EA
S1139280FFF7D4FF002002BD10B514460A4621465C
S1139290BDE810400123F7F7EBB8FFF7FEBFC04667
S11392A0C046C046C046FFF7DBFD19E050F8041B7A
S11392B0CB0744BFA9F101035918121F0023042A44
S11392C041F8043BF9D25FEA827C0B4604D54FF0A7
S11392D0000CA1F800C09B1CD10744BF00211970E9
S11392E050F8042B002AE1D170470000BFFFFFFFB4
S11392F0200500000004FF1F2C0F00002009FF1FA1
S10793000000000065
S9030411E7
